:020000040800F2
:10000000381100200101000817380008A528000851
:1000100015380008350F00083D6400080000000096
:100020000000000000000000000000006D49000812
:10003000731A000800000000853D00086D4C0008A0
:100040001B010008793B00081B0100081B01000888
:100050001B0100081B0100081B0100081B01000810
:100060001B0100081B0100081B0100081B01000800
:100070001B0100081B0100082D1500081B010008CA
:100080001B0100081B0100083D0700081B010008B8
:100090001B0100081B0100081B0100081B010008D0
:1000A000DD4C0008C94D00081B0100081B010008B9
:1000B000CD4D0008BD500008195300081B01000871
:1000C0001B0100081B0100081B0100081B010008A0
:1000D0001B010008355F00081B0100081B01000818
:1000E0001B0100081B0100081B010008DFF80CD0F1
:1000F00000F0E6FA00480047AD750008381100200E
:100100000648804706480047FEE7FEE7FEE7FEE7B1
:10011000FEE7FEE7FEE7FEE7FEE7FEE78D4C0008A0
:10012000ED0000082DE9F0410024061B254671F181
:10013000000605DA01240027D0EB070067EB010178
:10014000161E73F1000605DA0027D2EB070201251F
:1001500067EB030300F0D0F986460E4617469C462F
:10016000AC4204D00025D0EB050E65EB010624B1AE
:100170000020D2EB000760EB030C704631463A4694
:100180006346BDE8F08140EA01039B0703D009E024
:1001900008C9121F08C0042AFAD203E011F8013B73
:1001A00000F8013B521EF9D2704780EA010210B5F7
:1001B00002F00043400022D04A001FD0010E01EBA4
:1001C0001261C0F35600C2F3560240F4000042F43C
:1001D0000002A0FB022000047F39140400D0401C60
:1001E00050EA124001D44000491EC2B20C0604EB92
:1001F000D010401C4008802A02D003E0002010BD2F
:1002000020F00100002900DA0020184310BD2DE97C
:10021000FE4F81EA030404F0004421F00041009401
:100220004FF0000B23F0004350EA01045ED052EA85
:1002300003045BD0C3F30A54C1F30A552C44A4F25F
:10024000F3340194A0FB0254C1F3130141F4801173
:10025000C3F3130343F4801301FB024400FB034E7A
:10026000840A970A44EA815447EA8357A4FB076843
:1002700002958D0A05FB07854FEA932C04FB0C546D
:100280002705029D4FEA065847EA1637B5EB0805E1
:100290006EEB070C870E920E47EA811742EA831233
:1002A000A7FB0201B6EB0B0164EB00042B0D43EA44
:1002B0000C335E1844EB1C50DA465146E7FB020152
:1002C000C5F313044FEA0B3343EA14534FEA0432E5
:1002D000019C43EA0603A4F10C040294009CCDE9BE
:1002E00000B400F09FF903B0BDE8F08F0020014694
:1002F000F9E72DE9F04D81EA030404F0004B21F009
:10030000004514464FF0000A23F0004150EA050270
:1003100020D054EA01021DD0C5F30A570246C5F3A6
:100320001303C1F31300C1F30A5640F4801543F4DC
:100330008013A7EB0608101BD64608F2FD3873EBB6
:10034000050002D308F1010801E092185B41B8F101
:10035000000F03DA00200146BDE8F08D00204FF4C5
:100360008011064684460EE0171B73EB050705D384
:10037000121B63EB050306434CEA010C49084FEAE4
:10038000300092185B4150EA0107EDD152EA0300B8
:1003900012D082EA040083EA0501084305D0101B4D
:1003A000AB4106D20122002306E000224FF00043B9
:1003B00002E06FF0010253101AEB06004CEB0851FB
:1003C00010EB0A0041EB0B01BDE8F04D00F01BB94A
:1003D00070B521F0004303430CD0C1F30A5500244B
:1003E000D5EB040564EB0403D617AD1AB34102DB69
:1003F0000020014670BD201841EB025170BDC10FB5
:1004000080EAE0700844CA079623002100F0CDB8C6
:1004100096230022114600F0C8B80EB5C10F80EA3D
:10042000E0700844CA07002140F233438DE80E0013
:100430000A460B4600F0F6F803B000BD0EB540F2D8
:10044000334102910021CDE900110A460B4600F02C
:10045000E9F803B000BD00F0004220F00040C10DFB
:10046000C0F3160040F400007F2901DA0020704735
:10047000962903DCC1F19601C84001E09639884015
:10048000002AF4D04042704770B5C1F30A5201F01F
:1004900000450024C1F3130140F2FF3341F4801101
:1004A0009A4201DA002070BD40F233439A42A2F230
:1004B000334203DC524200F05FF800E090402C43EE
:1004C000F1D0404270BDC1F30A5210B5C1F313011F
:1004D00040F2FF3341F480119A4201DA002010BD4E
:1004E00040F233439A42A2F2334203DC524200F01C
:1004F00043F810BD904010BD2DE9F05F0546002087
:1005000092469B4688460646814640241BE0284684
:1005100041464746224600F02FF853465A46C01A35
:10052000914110D311461846224600F016F82D1AB4
:1005300067EB01084F4622460120002100F00DF82C
:1005400017EB00094E41201EA4F10104DFDC4846F0
:1005500031462A464346BDE8F09F202A04DB203A74
:1005600000FA02F1002070479140C2F1200320FA06
:1005700003F3194390407047202A04DB203A21FA04
:1005800002F00021704721FA02F3D040C2F12002AC
:1005900091400843194670470029A8BF7047401C86
:1005A000490008BF20F00100704710B4B0FA80FC89
:1005B00000FA0CF050EA010404BF10BC704749B1C6
:1005C000CCF1200421FA04F411FA0CF118BF012136
:1005D00021430843A3EB0C01CB1D4FEA00614FEA16
:1005E000102042BF002010BC704700EBC3501044E5
:1005F0000029A4BF10BC7047401C490008BF20F070
:10060000010010BC704710B5141E73F1000408DA25
:10061000401C41F1000192185B411A4301D120F0C6
:10062000010010BD2DE9F04D92469B4611B1B1FA83
:1006300081F202E0B0FA80F220329046FFF78DFF9F
:1006400004460F4640EA0A0041EA0B0153465A4667
:10065000084313D0114653EA010019D0C8F14002F3
:100660005046FFF789FF05460E465046594642461A
:10067000FFF773FF084305D0012004E02046394608
:10068000BDE8F08D0020054346EAE0762C43374371
:100690000A986305E40AA0EB08000022FD0A44EA78
:1006A00047540A3002D500200146E9E70105101938
:1006B0006941DDE9084500196941BDE8F04DA2E74F
:1006C000064C074D06E0E06840F0010394E807009F
:1006D00098471034AC42F6D3FFF70CFD9898000809
:1006E000B898000870B58C1810F8015B15F0070376
:1006F00001D110F8013B2A1106D110F8012B03E0BB
:1007000010F8016B01F8016B5B1EF9D12B0705D4C2
:100710000023521E0DD401F8013BFAE710F8013B0B
:10072000CB1A921C03E013F8015B01F8015B521E27
:10073000F9D5A142D8D3002070BD000070B54C4C53
:100740004FF490652946204600F015FA002864D041
:100750002946204600F0A2F846490888401C088037
:100760000121204600F0E6FA434942F21072B1F846
:100770005800904202D2401CA1F8580007F0FAF845
:100780003E4DB5F91410B5F9120005F0BBFF3C4C15
:10079000A5F856002080A16820468847A088A5F8C3
:1007A000580003F0A1F807F0E1F9364E364C3078E6
:1007B000082833D045F6AC30606042F6EF60A060A8
:1007C00042F2C400E0603148008A2080208E6080C0
:1007D000A16B2D488847208E69882D4C08444FF620
:1007E000FF7101EA80006887207A4FF0000540071A
:1007F0001DD501F0CDFA274949F6A24008802648C8
:1008000040F21A62C188491C89B2C180914204D366
:10081000A16821F00401A160C58070BD41F2130000
:1008200060604FF48060A06040F61B50CAE73078EB
:100830000A2818D2DFE800F0170613050A050D177D
:100840001113EAE7BDE8704006F006B908F05EF95A
:1008500005E0BDE8704002F091BD06F083FCBDE804
:10086000704007F0DBBA00F0FDFB84F8B65070BDB5
:10087000002401402C0700204801002064000020D3
:100880004C07002023070020E40000200002002085
:10089000AC020020442C01406C0900206FEA1121B9
:1008A000016070470029816802D041F0010101E038
:1008B00021F00101816070470029816802D041F474
:1008C000807101E021F48071816070472DE9F04171
:1008D000824E92B0304600F00BF90BA800F039FAC6
:1008E00001214FF4C06003F0E1FA00248DF831409B
:1008F0004FF46020CDE90D044FF4A0204FF009081B
:100900000B9001278DF83C808DF830700BA9304694
:1009100000F080F9724D8DF831408DF830708DF80F
:100920003C700BA9284600F075F901231A460F21E7
:10093000304600F0C0F9022201231146304600F093
:10094000BAF9012303220021304600F0B4F9012353
:1009500004221946304600F0AEF9012305220B218E
:10096000304600F0A8F9012306220421304600F0A9
:10097000A2F9012307220821304600F09CF9012347
:1009800008220321304600F096F9012309220A21AA
:10099000304600F090F90121304600F084F9012141
:1009A000284600F080F901231A460521304600F060
:1009B00055F901231A460621284600F04FF9002177
:1009C000304600F0CBF84FF4E041284600F0C6F87E
:1009D0000121304600F0B8F80121284600F0B4F8B3
:1009E0000121304600F0A6F80121284600F0A2F8C7
:1009F0000121304600F09EF90121284600F09AF9C5
:100A000040F61451374804F05EFF12208DF8400084
:100A100002208DF841008DF842408DF8437010A8F7
:100A200002F026FF01224FF49061304600F0E8F812
:100A300001213046FFF740FF01213046FFF732FF2A
:100A400001212846FFF72EFF304600F06EF93046B0
:100A500000F09FF80028FAD1304600F075F93046D2
:100A600000F082F80028FAD1284600F05EF9284606
:100A700000F08FF80028FAD1284600F065F92846E2
:100A800000F072F80028FAD10121084603F0EAF9D3
:100A9000154D284600F086FD684600F02EFE0F48F2
:100AA00001A94C300090114881E811018020CDE966
:100AB00004404000069080000790202008904FF4EA
:100AC0004050CDE909046946284600F0F9FD0121AE
:100AD000284600F05BFD12B0BDE8F0810024014023
:100AE00000280140002C014008000240BC02002008
:100AF0000D4910B5884202D1012144150AE00B4985
:100B0000884202D10121041504E0094988420AD132
:100B10000121CC03204603F0D5F92046BDE8104062
:100B2000002103F0CFB910BD00240140002801408E
:100B3000003C01400029816802D041F4801101E0AD
:100B400021F48011816070470029816802D041F44E
:100B5000004101E021F4004181607047826822F485
:100B6000E0420A43826070470146002089684907D5
:100B700000D50120704710B50246002054680B0ACA
:100B8000C9B20C401168194202D0002C00D00120DB
:100B900010BD014600208968090700D50120704773
:100BA00038B501211C2003F081F9FF20ADF80000C9
:100BB00000248DF8034003258DF8025069460D4846
:100BC00001F0E0FA0120ADF800008DF803408DF847
:100BD00002506946084801F0D5FA2320ADF800001C
:100BE0008DF803408DF802506946044801F0CAFAB6
:100BF00038BD000000080140000C01400010014019
:100C0000002A4268C9B201D00A4300E08A43426028
:100C10007047000010B542680E4B0C791A400B6803
:100C200042EA04221343436083680B4A1340D1E92C
:100C3000024222434C7943EA44031A438260C26A67
:100C4000097C22F47002491EC9B242EA0151C16214
:100C500010BD0000FFFEF0FFFDF7F1FF70B50724A7
:100C600009290AD9C568A1F10A0606EB4606B4406F
:100C7000A543B3401D43C56007E0056901EB41068C
:100C8000B440A543B3401D430561836BC3F30154D6
:100C9000121B921C02EB82041F22A2409343A1402C
:100CA0000B43836370BD826B491E22F4401242EAFB
:100CB00001518163704770B5072409290AD9C568B5
:100CC000A1F10A0606EB4606B440A543B3401D4316
:100CD000C56007E0056901EB4106B440A543B34098
:100CE0001D4305611F23072A09D2446B521E02EBE4
:100CF000820293409C4391400C43446370BD0D2A93
:100D000009D2046BD21F02EB820293409C439140B4
:100D10000C43046370BDC46A0D3A02EB8202934037
:100D20009C4391400C43C46270BD816841F008014E
:100D3000816070470029816802D041F4A00101E080
:100D400021F4A00181607047816841F00401816055
:100D5000704700210160017141718160C160012112
:100D60000174704770B51E4C214694F83800B1F8F4
:100D7000425006281ED9B4F84A10B4F84C00A1EB32
:100D8000000202F10902122A04D8FFF757FB0022E1
:100D9000144B0AE0884204D2FFF750FB0022124BAA
:100DA00003E0FFF74BFB0022104BFFF730FAFFF791
:100DB0008AFB09E005D12846FFF740FB0C4A0D4BA2
:100DC000F3E70D4951F82000C5EB45116063B0EB26
:100DD000410F03D9C5EB45104000606370BD0000B2
:100DE000580400200000344000003340000035402B
:100DF0006766666666E64B40488F000810B50C4C87
:100E00002078400713D5FFF7ADFF0A49A08E088070
:100E100008483038018821F010010180001F018846
:100E200041F010010180207820F00400207010BDF6
:100E30005804002040040040F0B4184816494FF40C
:100E40009677436C08468A68046815485FEAC25C76
:100E500042F00806007822F008054FEA047415D520
:100E6000002C08DB120714D408B1082811D1BB42AA
:100E70000FDA8E6007E012070BD508B1082808D1F9
:100E8000BB4206DA8D60F0BC05F06EBF002CF2DAD2
:100E9000E8E7F0BC70470000AC02002048010020E9
:100EA0002307002070B506464089204B204C4FF4A4
:100EB0008071002580B362887AB1012A0CD1E18863
:100EC000491C89B2E1803289914205D36580E58071
:100ED000FF2801D0401E708170BD7088228890422A
:100EE00001D9012200E00022184601F0D4F97088EF
:100EF000B18801442088401C80B220808142EBD818
:100F00002580A088401C80B2A080F1888842E3D36D
:100F100001206080A58070BDFFE70022184601F027
:100F2000BAF9A580E58025806580F4E7000C0140D2
:100F3000C8050020FEE70000FCB505464FF6FF7629
:100F400000200C46ADF8006048F205078DF804005B
:100F500020E000BF15F8010B8DF8040001A9084638
:100F600002F0C9F8BDF800009DF8041080EA0120E5
:100F7000ADF800005FF00000BDF800100A0402D5D3
:100F800087EA410101E006EA4101401CADF800108A
:100F90000828F1DB641EDDD26946084602F095F8A8
:100FA000BDF80000FCBD00000246002004E000BFC8
:100FB00012F8013B1844C0B2491EF9D27047000034
:100FC00070B5144A85B01088002413490194009428
:100FD000039420460494138807E00D8B009E35444B
:100FE0000095CD8B019E3544019515889D42F4D026
:100FF000401CC0B28028EED30098411107484180C0
:10100000848001984111064881830183818205B063
:1010100070BD00002C070020AC020020E20500207B
:10102000D004002030B50E4902880A800C4A43885B
:10103000083A13800B1F808818802024151F2C80ED
:101040000020401C80B27328FBD341F211100880AD
:1010500044F64800108047F2480018802C8030BDCC
:10106000202C0140114944F648000880091D46F62D
:1010700048000880091D41F2111008800B48001F2C
:10108000018841F02001018009480021A0F8641086
:10109000A0F86210A0F86010A0F85E10A0F85C1034
:1010A000A0F85A100348418181827047182C0140F2
:1010B000AC020020640000202DE9F04F524B534851
:1010C0000022D97A90F800C080292CF001067DD347
:1010D0001C684F4B01F01F0153F821104D4B0C427F
:1010E000196802D041F0200101E021F02001994669
:1010F0001960484BDFF820B1DFF820A193F8465083
:10110000474B9BF80040B3F90430022C69D1B9F881
:101110000840C4F3C007C4F30024A74261D03D4C8B
:101120002C3C94F80380B8F1000F09D0374FB8F188
:10113000010FB7F902700DD0B8F1020F56D120E0BF
:101140000A0553D58A0651D40122E2702CF004021C
:1011500002704BE00E0549D48E0647D55FEA4C7607
:1011600044D4A7BB4380002B09DD4CF0050202707C
:101170000222E2702B4AB2F84420028236E0E2708A
:1011800034E0B0F806C0BCF1000F01D1002B17DC31
:1011900090F80CC0AC4513D107F26667BB420FDC78
:1011A000214FBF895FEA477C0AD45FEA877C07D476
:1011B0005FEA417C04D55FEA816C01D5FF0715D059
:1011C00006704280AAF80020428101E017E00DE09D
:1011D000426182610282E27089F80F208BF8002060
:1011E00004E006704280AAF800204281C3800573A3
:1011F000480960F3CB21C9F80010BDE8F08F0670F4
:1012000042804281F9E70000E805002050090020F3
:10121000A8930008AC02002023070020240100202E
:10122000E205002048010020600A00202DE9F04777
:1012300096B000240C940D940E940F9472B69048BE
:10124000816941F400718161816941F4806181614A
:101250004FF4004002F0FCFD8A4D00212846FFF7C4
:101260002BFB00212846FFF71DFB874E002130464F
:10127000FFF718FB854F0021384600F087F9012061
:101280004FF47041401C8842FCD32846FFF730FCE5
:10129000B1463046FFF72CFC384600F083F94FF496
:1012A0006020CDE912048DF8454001204FF004087C
:1012B0008DF8440010948DF8508010A92846FFF74F
:1012C000A9FC01231A4605212846FFF7F4FC012357
:1012D000022206212846FFF7EEFC01230322072104
:1012E0002846FFF7E8FC012304220F212846FFF7D8
:1012F000E2FC384600F056F9684600F0FEF9614815
:10130000634E4C300090CDF80C80CDE90164802014
:10131000CDE904404000069080000790202008900E
:101320004FF44050CDE909046946384600F0C8F949
:1013300001212846FFF7C0FA0121384600F026F9BE
:1013400001212846FFF7AEFA47F23051159415985F
:10135000401C15908842FAD301212846FFF7EAFC89
:10136000ADF82C40A04640F2DC5A4FF4007420E067
:101370005046CDF854801599491C15918142FAD3F5
:1013800030880D9908440D9070880E9908440E908D
:10139000B0880F9908440F90F0880C9908440C907D
:1013A00001212846FFF7C6FCBDF82C00401CADF813
:1013B0002C00BDF82C00A042DAD30D98354A40F33A
:1013C000CF1633480A3006830E9941F3CF14448375
:1013D0000F9941F3CF1383830C9941F3CF1CA0F8ED
:1013E00004C0ACF5C05C40F2C371ACF59B7C8C458D
:1013F0000ED2A6F5C856363E8E4209D2A4F5C85480
:10140000363C8C4204D2A3F5C853363B8B4203D3FF
:10141000D18841F48041D180D188490407D41E4944
:10142000028B21F85C2F428B4A80808B88800021C0
:101430002846FFF741FA0021384600F0A7F80021BE
:101440002846FFF72FFA00214C464846FFF72AFAB4
:101450000220C102401C8842FCD32846FFF748FB0B
:101460002046FFF745FB384600F09CF8FFF72EFAC0
:101470000A493C20087062B616B0BDE8F08700004B
:1014800000100240002401400028014008000240F2
:101490002E050020600A0020C00C0020200700203C
:1014A00070B5204B40F6C81441F2B7055B6C48F6A6
:1014B000E6065C4305EBA4341B4D73434EF6F6166B
:1014C00006EBA333C5E90443D460401A53611060AE
:1014D0009168884202DA4942884200DC1160106853
:1014E0004343107E0341906A19189162506A814209
:1014F00000DD9062916A106A814201DB084600E0DB
:101500009062A86111684C43117C0C41084121187C
:10151000B2F91C00884204DBB2F91A00884200DCF0
:1015200008B270BD480100202801002010B54FF41A
:101530000054204600F0ACF8002813D00A4908787F
:1015400040F008000870204600F014F80021074819
:1015500000F01CF80648C17E012903D10021C176A4
:101560000121017710BD00008206002044000240E6
:10157000640B0020C10002D502490860704702498F
:1015800048607047040402400000024000290168DE
:1015900002D041F0010102E04FF6FE7211400160FD
:1015A0007047000001684FF6FE7211400160002193
:1015B000016041608160C1603149314A083990421F
:1015C00003D1486840F00F0006E02D4A14329042E3
:1015D00004D1486840F0F00048607047284A28323B
:1015E000904203D1486840F47060F5E7244A3C32E9
:1015F000904203D1486840F47040EDE7204A5032F1
:10160000904203D1486840F47020E5E71C4A6432F8
:10161000904203D1486840F47000DDE7184A783200
:10162000904203D1486840F07060D5E7154A111F19
:10163000904203D1086840F00F0006E0114A1432CE
:10164000904204D1086840F0F000086070470D4AED
:101650002832904203D1086840F47060F5E7094AE7
:101660003C32904203D1086840F47040EDE7054AEF
:1016700050329042EAD1086840F47020E5E700005B
:101680000800024008040240406880B27047000031
:1016900001460020CA0001D5034A00E0034A12684F
:1016A0000A4200D0012070470004024000000240BE
:1016B000002A026801D00A4300E08A4302607047B2
:1016C00030B5036847F6F07293430C6A8A68224388
:1016D000D1E904452C4322438C692243CC6922433F
:1016E0004C6A22438C6A22431A430260CA684260F1
:1016F0000A6882604968C16030BD002101604160B4
:101700008160C160016141618161C16101624162C9
:101710008162704710B5114C8CB000212046FFF754
:1017200035FF2046FFF73EFF0D4800900D48002191
:10173000CDE901016420CDE903018020CDE9050157
:101740000791089109910A9169462046FFF7B8FF71
:1017500001212046FFF71AFF0CB010BD58000240CF
:1017600004380140BC07002010B501218CB00846A8
:1017700002F078FB1E4C00212046FFF707FF2046B1
:10178000FFF710FF1B4800901B480190002110201C
:10179000CDE902018020CDE904100691079108915E
:1017A00009910A9169462046FFF78AFF012202212A
:1017B0002046FFF77DFF01218DF82F1004208DF8C2
:1017C0002D008DF82E100E208DF82C000BA802F0A5
:1017D0004FF80F208DF82C000BA802F049F80121DA
:1017E0002046FFF7D3FEFFF795FF0CB010BD0000B9
:1017F00044000240043801405807002030B540F64C
:10180000AA21204AC184838B1488E31A9BB20F2B30
:1018100010D312888283037E002253B11A4BB3F98E
:101820000A30062B05DB194B1B78022B03D0002B4B
:1018300000D1828430BD164B40F68B255B6CA3F241
:101840002D14AC420FD2428B521C92B24283642AB6
:10185000F0D364224283B0F924208A4201DA02EBF9
:101860002111818430BD41F29414A342FADBB0F916
:101870002430002B02DDA3EB211100E00021818444
:10188000428330BD2C070020640000202307002085
:101890004801002010B50446B0F9020043F6991142
:1018A00048438113E06840F26662504301EBA03088
:1018B000E060B4F9001043F6991251438A1321698C
:1018C00040F26663594302EBA131216104F0BAFE94
:1018D0006061A18840F6AB2208444010A0F5154194
:1018E0005539E062914205D9A0F5F851FF39521CF3
:1018F00091421DD249F25451884202DDA0F52040A8
:1019000002E0A0F5F850FF38206300EB400040F300
:101910004F002085B4F924104A42904201DA104663
:1019200002E0884200DD0846E083228461848AE088
:10193000A0F5FE42FF3A41F255518A4214D8A2F670
:10194000AA20206300EB400040F34F002085B4F94B
:1019500024205142E183884201DA084602E09042A5
:1019600000DD1046404250E0A0F5D442AA3A8A4237
:1019700015D2A2F6AA20206300EB400040F34F01ED
:101980002185B4F924004242E2832084914201DAA5
:10199000104602E0814200DC0846608453E0A0F576
:1019A000AA42543A41F256539A4215D2A2F6AB20BB
:1019B000206300EB400040F34F002085B4F9241071
:1019C0004A42904201DA104602E0884200DD0846B1
:1019D0004042E083218419E0A0F5804241F2545353
:1019E0009A4215D2A2F6AA20206300EB400040F3F1
:1019F0004F012185B4F92400E0834242914201DA8B
:101A0000104602E0814200DC0846208462841AE02D
:101A1000A0F52852AB3A8A4215D2A2F6AA2020633A
:101A200000EB400040F34F012185B4F92400E0832E
:101A300042422284914201DA104602E0814200DCF7
:101A400008464042A9E7B4F91E00A0EB40208013ED
:101A5000E080B4F92000A0EB402080132081B4F98D
:101A60002200A0EB40208013608110BD012101768F
:101A7000704770471548164A4FF480410078042893
:101A800021D002F13C03D08A9B88C01A00B22F28D3
:101A900001DD001108E0002801DD002007E00D4B0A
:101AA000984201DA184602E0402800DD4020938980
:101AB000184400B2884203DC40F26661884200DAD2
:101AC00008469081704791817047000023070020ED
:101AD000D0040020C0FEFFFF38B54B484B490288B8
:101AE0000B889A1A92B20F2A71D30988484C018048
:101AF0004FF0FF01E2884FF47A7355044FF496706B
:101B000002D51622009103E0950403D51522009119
:101B1000014670E0D50402D514220091F8E71505BE
:101B200002D513220091F3E7550502D51222009148
:101B3000EEE7950502D511220091E9E7D50502D51A
:101B400010220091E4E7150602D50F220091DFE78D
:101B5000550602D50E220091DAE7950602D50D2230
:101B60000091D5E7D50602D50C220091D0E71507E4
:101B700002D50B220091CBE7550702D50A2200912E
:101B8000C6E7950702D509220091C1E7D20702D026
:101B900008220091BCE72289550702D5072200914F
:101BA000B6E7950702D506220091B1E7D20702D029
:101BB00005220091ACE7A27AD20702D0042200915C
:101BC000A6E7A289D40603D503220091A0E719E075
:101BD000140702D5022200919AE7540703D4940710
:101BE00001D4D20702D00122009191E700200346E0
:101BF00002460146009002F065FFBDE83840024809
:101C0000FFF750B938BD0000540A00202C0700200F
:101C1000600A0020F0B55948594982880B889A1A01
:101C200092B29C2A64D30988818056490A88014669
:101C3000002A0B7843F0020156D11646524A1C077F
:101C400015680246127822F0020274D54F4C0746FE
:101C5000E4887F785FEA845C02D547F0010701E001
:101C600027F001074770A704477802D547F002071D
:101C700001E027F002074770670401D4E70703D0AB
:101C8000477847F008074770640603D5447844F066
:101C9000040404E01C0603D4447824F004044470D3
:101CA000EC0450D4354C9A07247824F0100423D443
:101CB000324D42782F7A2D78012A45F0100514D044
:101CC000022A16D02D4C042AA47804F1010C0CF041
:101CD000FF0C13D0072A25D0032A23D0052A21D0B0
:101CE000062A1FD021F0100142E0B90702E005707A
:101CF000F0BD39070029FADB0470F0BDFA0601D403
:101D00001A060AD50170022C04D280F802C0BCF178
:101D1000020FF2D341F080012AE021F0100101709E
:101D20008670F0BD877A7F06F7D5032C04D8017042
:101D300080F802C0F0BD0FE05107D8D51906D6D4FF
:101D400043F0800114E002704178CB0701D189078C
:101D5000F0D522F010010BE0E9040BD49907E9D487
:101D6000818AC82902D2491C8182E3E743F00A0133
:101D70000170DFE702708682DCE7000004070020C4
:101D80002C0700202E070020AC020020600A002053
:101D9000094944F648000880091D46F648000880B5
:101DA000091D41F6CC4008800348001F018841F01E
:101DB0002001018070470000182C0140084946F6B8
:101DC00068000880091D0880091D41F255500880EF
:101DD0000348001F018841F0200101807047000086
:101DE000182C014010B5C28800210AB1032206E078
:101DF00002890AB1022202E0428912B10122027074
:101E000000E0017004784FF4804344F6206244B14E
:101E1000012C06D0022C07D0032C01D141808180F7
:101E200010BD4380828010BD41F23331418040F6C5
:101E3000B731F4E730B5B1F86A5000231A240D2207
:101E4000854202DCB1F9680030BD4D88854202DB75
:101E5000B1F9000030BD01EB82056D88854201DDDE
:101E6000144601E013DA134604EB03024FEA520270
:101E70009A42F0D101EB830231F823105488928802
:101E8000521A001B424301EB622000B230BD31F90F
:101E9000220030BD054920B1086940F0800008618A
:101EA000704703484860034848607047002002407C
:101EB00023016745AB89EFCD06494FF47A70CA68B4
:101EC000D20705D0401E0004000CF8D1FF20704757
:101ED00000207047002002400E4A0320A2F150016A
:101EE00082F83E00002048810B490886C862C883FA
:101EF0000884488490620948016DB1F5206F01DBC8
:101F0000A3219162807A002802D0906A40429062B8
:101F100070470000640000203805002048010020C0
:101F20000449002048810881C862886202498862A9
:101F30007047000064000020CC080020F0B53B4949
:101F400088894A89801A80B20F2866D38889488197
:101F5000CA8937480B3A272A26D28A7822BB826858
:101F6000364B42F480728260324A354C354D1278DD
:101F70005607314A0AD4344E36881680334A1288BE
:101F80001A80334A12882280324A09E0324E36885B
:101F90001680324A12881A80314A12882280314AC9
:101FA00012882A8001228A702F4B304D19469A7F61
:101FB0000968802A32D302F01F0255F8222011420C
:101FC0002CD0826822F48012184E82601236144699
:101FD0001215B778521C62F38617254AB77093F82A
:101FE00016C01778BCF1800F27F0020608D30CF05A
:101FF0001F0C55F82CC011EA0C0F01D147F0020656
:1020000016701A7E802A0DD302F01F0255F8222086
:10201000114207D144F400218160F0BD826842F48E
:102020008012D1E724F40021F6E700002007002009
:10203000AC02002048010020C8040020CA0400208F
:10204000CC040020CE040020B8040020BA040020F4
:10205000BC040020BE040020C0040020C2040020F4
:10206000C4040020C6040020E8050020A89300084E
:10207000D004002070B5204881890289891A89B26C
:102080000F292FD3818901811C4B1D4819465D7A88
:1020900006681C4C096846F00402802D07D305F041
:1020A0001F0554F82550294201D126F00402026090
:1020B0009A7B802A17D302F01F0254F82220114283
:1020C00011D1026822F002020260DA7A802A0ED36D
:1020D00002F01F0254F82220114208D1016821F0B9
:1020E0000801016070BD026842F00202ECE701687D
:1020F00041F00801F5E7000020070020E805002076
:10210000AC020020A8930008F0B51D4C1B4A4FF00C
:10211000010C94F83B5094F80AE0144692F83C30D5
:1021200094F838402B43651CEEB2154D95F83D7080
:102130000025BEF1FF0F0AD0BEF1000F06D18B4281
:1021400013D155700C2C01D282F83860F0BD834257
:1021500002D182F801C0F5E78B42F7D15570B8077C
:1021600009E000BF82F83850F0BD8342FCD1F8434B
:1021700082F801C080070028F4D0F0BD5804002088
:1021800048010020F0B5CA78002502F00F03D206FE
:1021900001D58A7813430A784FF00F0E12F0FF0F23
:1021A0004FF001021CD004680F8802FA05F6374090
:1021B000B74211D14FEA850C0EFA0CF724EA070753
:1021C00003FA0CF43C43CF78282F02D0482F02D0DA
:1021D00002E0466100E006616D1C082DE4D3046056
:1021E0000C88FF2C1ED944685FF0000606F1080732
:1021F00002FA07F50F882F40AF420FD14FEA860C45
:102200000EFA0CF7BC4303FA0CF73C43CF78282FA7
:1022100000D14561CF78482F00D10561761C082E8A
:10222000E4D34460F0BD0000F0B5144C002801DA9E
:10223000E36900E06368420D120185B2C0F3015703
:102240009540C0F30346032F05D0C2020AD50322EE
:10225000B240934307E023F07062636823F0706339
:10226000636002E0AB4343F0706201B12A4300288F
:1022700001DAE261F0BD6260F0BD000000000140E3
:102280000246002092680A4200D001207047416156
:102290007047016170470AB1016170474161704741
:1022A0000F4A104B92F838105B5C834201D1012039
:1022B00004E00D4B5B5C834203D1002082F83A00BE
:1022C00070470A4B5B5C834201D18120F6E7084BE3
:1022D000595C814201D18020F0E70320EEE7000045
:1022E000480100206098000872980008669800086D
:1022F000789800080A4810B501784FF000024C07A2
:1023000008494FF0FF0389684FEA017105D500299C
:1023100001DA827210BD837210BD0029FBDBF8E781
:1023200048010020AC020020F0B5194E194C0022E3
:10233000E31CA6F1060CB75CA518ED78FF5C0D4315
:102340000F43BD421FD01CF80270FF5C0F43BD421B
:1023500019D015460023A618F6780E43C6545B1C08
:102360001CF80220DBB2062BF5D3C178817001790D
:10237000C17000214218491C15711CF80550C9B2E2
:102380000629F7D3F0BD521CD2B2032AD3D3F0BD35
:102390003A8F00085804002010B502460021064B71
:1023A00006205C186478944200D10846491CC9B2E2
:1023B0000629F6D310BD000048010020214810B5C1
:1023C00090F8671000222048012936D11F498988DA
:1023D00099BB1F491E4B4C6C40F6B831B3F87630B0
:1023E0008C4227DD1B49097821BB90F82711491C35
:1023F000C9B280F82711C8291CD380F827210146CB
:10240000D0F82C4191F82811A34203DD052908D208
:10241000491C01E041B1491E80F82811C9B20529C3
:1024200002D3012180F82611191B074C2C3C616254
:10243000C0F82C31B3F5FA6F03D280F8262180F86A
:10244000282110BDC00C0020AC020020E2050020B5
:1024500048010020230700204FF4C042C260002141
:1024600081620E22028241F26202426108220283EC
:102470004FF46042428381834FF07842C0E90821E3
:1024800040F6C41101807047B0F90010B0F9022085
:10249000891A41604269037E4A431A41836A1344A0
:1024A0008362426A934200DD8262836A026A9342D7
:1024B00000DA8262C268836A4A43017C0A410B41A6
:1024C000D118B0F91C208A4201DA10467047B0F9E1
:1024D0001A008842FADC08B27047000010B51448B0
:1024E0001449B0F894200B889A1A92B2B2F5437F3F
:1024F0001DD90988A0F89410B0F8921020F8601F38
:10250000002242860C480D4CC2888280C180C3895B
:1025100083812489891AA4B2C4818160E11A01618E
:10252000074A818AC182928A8282511A816110BDD2
:10253000480100202C070020880C002038050020CE
:102540006400002009480A49B0F8B2200B889A1AA2
:1025500092B241F684639A4206D3098820F8B21FEA
:10256000418881800021418070470000480100209F
:102570002C0700200D480178C90702D00C490988B2
:1025800001E04FF6FA7141660949012010390880CF
:1025900007482438018841F00101018004481838B7
:1025A000018821F0180101807047000048010020D7
:1025B000240400400A49D1F8982012B1521EC1F8F3
:1025C000982031F8922F521C21F81A294A6A521C7D
:1025D0004A628A8F521C8A8701F8400C70470000BB
:1025E000480100201CB52D4890F83B3090F83C2065
:1025F000934252D000248DF8044053408DF80030AF
:102600009DF800300122012B08D09DF80030022BEC
:1026100009D09DF80030042B0AD00DE01F498DF839
:102620000420443108E01D498DF80420463103E0C0
:102630001A498DF8042048319DF80420012A2CD134
:1026400090F83D309DF80040154AA34217D090F80D
:102650003E309DF80040234208D0B0F84C30A0F83E
:102660004A300B881488E31AA0F84C3090F83830C0
:102670002BB1B0F840301488E31AA0F84230128829
:102680000A80A0F8402010F83E1F9DF8002011435A
:1026900000F801199DF8001001701CBD58040020BD
:1026A0002C07002070B5344D40212846FFF7E8FD87
:1026B000840080212846FFF7E3FD44EA4004A91581
:1026C0002846FFF7DDFD0443E1B22C4C94F8785026
:1026D0008D4250D04D4084F87810012D03D0022D4A
:1026E00001D0042D47D194F87C00A84384F87C00E5
:1026F00094F87B20AA420FD084F87B5094F87A207B
:1027000001238B401A4207D11A4384F87A2094F8A7
:102710007910491C84F8791094F87910042928D389
:1027200030B1012811D002280FD004280DD012E0BA
:102730001348C18821F04001C1802078002184F82D
:102740003B1020F06000207005E0217841F020016E
:10275000217084F83B000B4994F83B0091F8272046
:10276000904204D081F8270007492020087000F02B
:102770000DF884F8545070BD00100140480100204D
:10278000600A0020C00C00202007002070B50D4D0D
:1027900040212846FFF774FD840080212846FFF77A
:1027A0006FFD44EA4004A9152846FFF769FD04437C
:1027B0000548072100F8784F0171002141708170B0
:1027C000C17070BD001001404801002070B5344850
:1027D00090F83A10CA43920761D001F0030280F8E2
:1027E000392090F83D305B061B0E80F83D30012A01
:1027F00001D0812A02D15B1C80F83D300278D207DB
:102800004DD0DBB203F00102C3F34004A24246D133
:10281000B0F856400025641CA0F85640204CA0F8A3
:10282000585090F83E60A47AB24202D080F83E2020
:102830000DE0A607B6EB837F02D080F83F5006E09C
:1028400090F83F30642B02D25B1C80F83F3090F848
:102850004030642B0CD25B1CDBB280F84030022B82
:1028600006D204F00103934202D1022280F84020F4
:10287000012901D0002912D190F83820416E00EBD7
:10288000820291610163D0E906121144D0E9082364
:102890001A441144826A1144C26A1144416370BDF2
:1028A00048010020FEE700002DE9F04F00BF0020A6
:1028B0009E4E9F4AA6F51271A6F5BE79A6F1440B6D
:1028C00006F1440E804601F5E074A1F1780301F5AC
:1028D000457A1D5C15F0C00706D0402F51D0C02F9F
:1028E00077D0802F76D004E115F01F0504D0154471
:1028F00040F080072F7201E082F80880012826D07E
:10290000022824D0032822D0042820D008281ED052
:1029100010281CD0874D55F820C0DCF8005054F822
:1029200020703D40CCF80050824D55F820C0DCF8B6
:10293000005056F820703D43CCF800501D5CAD06A9
:1029400059F820502F6813D53AF810C03EE051F8DE
:1029500020502F6854F820C007EA0C072F6051F868
:1029600020502F6856F820C047EA0C072F60E5E793
:10297000DFF8B8C10CF1F00C5CF820C007EA0C07D6
:102980007EE015F01F0504D0154440F080072F723B
:1029900001E082F8088001281DD002281BD00328FE
:1029A00019D0042817D0082815D0102813D0614D4D
:1029B00055F820502F6854F820C007EA0C072F6004
:1029C0005C4D55F820502F685BF820C047EA0C0793
:1029D00056E00BE056E051F820502F6854F820C024
:1029E00007EA0C072F6051F82050ECE715F01F059F
:1029F00005D0154440F0800785F8217001E082F889
:102A00002180012825D0022823D0032821D00428A2
:102A10001FD008281DD010281BD0464D55F820C0C7
:102A2000DCF8005054F820703D40CCF80050414D87
:102A300055F820C0DCF800505EF820703D43CCF81B
:102A400000501D5CAD0615D53A4D3AF81070CC35E6
:102A500014E051F820502F6854F820C007EA0C0702
:102A60002F6051F820502F685EF820C047EA0C070D
:102A70002F60E6E72D4D3AF81070E03D55F82050F4
:102A80002F6036E015F01F0505D0154440F0800793
:102A900085F8217001E082F82180012830D00228D9
:102AA0002ED003282CD004282AD0082828D010287B
:102AB00026D0204D55F820C0DCF8005054F8207086
:102AC0003D40CCF800501B4D55F820C0DCF80050BC
:102AD000164F883757F820703D43CCF800501D5CE6
:102AE000AD06B1D4114F3AF81050E03F57F82070BE
:102AF0003D60401CC0B21128FFF4EBAEBDE8F08F82
:102B000051F820502F6854F820C007EA0C072F60B6
:102B100051F820502F68DFF814C00CF1880C5CF8D5
:102B200020C047EA0C072F60D9E700003496000860
:102B3000E8050020309400084FF40771C1824FF47B
:102B40005861018340F6145181837047F0B5C48AFF
:102B5000B0F900608681B0F90250C581B0F9043047
:102B60000227002101220382AB4204DBB54202DDD1
:102B7000C78042810CE0B34204DBAE4202DDC78075
:102B800041811CE09D4205DBB34203DDC2804781E9
:102B9000018115E0B54204DB9E4202DDC280418125
:102BA00005E0AE4205DB9D4203DDC1804281078125
:102BB00006E09E4204DBAB4202DDC1804781028118
:102BC000C388458900EB430700EB4505BB89AE8907
:102BD0009B1B0FFA83FEA0F812E00689AB8900EB7D
:102BE000460CBCF80CC0A3EB0C038382B0F9183080
:102BF000B7F90CC0A3EB0C0CB4EB4C0F04DA80F863
:102C00002010A3F1A10113E0A64503DD80F82010F8
:102C1000B9890BE026B1012E04D0022E10D004E0B9
:102C2000062100E0052180F82010A989091B6D31DB
:102C3000418309B2B1F5586F04DB5B1E438304E0A6
:102C40000421F0E7002900DC4283418B8183F0BD41
:102C50000B49002288760A62CA614A62094A32F93F
:102C6000103002EB40028B62B2F90220CA62064ABF
:102C700032F810000882A1F86000A1F862007047E5
:102C8000000200208A9800087E9800082DE9F05F75
:102C9000FC48FD4982880B889A1A92B20F2A44D3C5
:102CA0000988FA4A8180814611880124F848F94E42
:102CB000002579B3491E1180C573F74A8562016802
:102CC000B2F902204F0742F6AA2318D4F78847F436
:102CD0000057F780F04E3678B60709D5866826F09B
:102CE00080068660A0F87C5080F87E5080F87F5087
:102CF000CE0404D480F8F040C0F8EC5003E080F833
:102D0000F0504E0707D49A4205DB80F8F440A0F853
:102D1000F25004E010E080F8F4504E0703D49A42D9
:102D200001DBC90703D080F81151BDE8F09F80F89E
:102D30001141A0F81251F8E78046B0F8181143F697
:102D40009820814202D2491CA8F8181101F0D0FE47
:102D5000D24FDFF830B397F85000ABF11C0B10B135
:102D6000FEF7AAF905E09BF8001021F001018BF8AD
:102D70000010FFF723FB00F0D5F9C94841F26802C3
:102D80004FF40061406C904201DBC64A04E0B0F5AC
:102D90007A6F02DAC34A121D116097F85110DFF8FA
:102DA000F0A2C14BC14FC907AAF12C0A3AD0997BB6
:102DB000802933D398F8002092072FD498F80F2059
:102DC0008AF80620B44A514692F800C02CF0020C52
:102DD00082F800C0ABF80250CBF814509BF800C04A
:102DE0002CF0010C8BF800C0B279520611D44A893C
:102DF000B2F5FA7F03D2521CAAF80A2012E040F67C
:102E00003C72904201DD002013E108208AF8044062
:102E10000FE10D710020AAF80A500AE18AF8045067
:102E2000AAF80A50D8F80800010501D5082000E1E9
:102E30009A4991F83FE05FEACE7149D09A4B98F8F1
:102E40000F208AF806205B7A4146802B4CD30B7802
:102E50005B0735D4F3889B0405D500BF20F0200024
:102E6000C8F8080034E0ABF80250CBF814509BF8D7
:102E700000C08D4B2CF0010C8BF800C040F02000FE
:102E80008860D87D80280AD300F07F0C1B684FF043
:102E9000004020FA0CF0034201D10C7100E00D71EA
:102EA0000879C00702D15FEA8E7005D50320032A96
:102EB00001D08AF80940BCE00020C8F82850B8E0EA
:102EC00020F02000C8F80800F08820F40050F080BE
:102ED00098F82601444601280BD0704890F863000A
:102EE00048B1FDF7A9FF0FE00A6842F004020A604A
:102EF000B4E709209DE0A068C10502D520F00800D4
:102F000001E040F00800A06094F846204FF48041B2
:102F1000E2B143F69913012A1FD0881E022A3A789B
:102F2000C2F381022CD0012A2FD0022A2DD0A4F87E
:102F300014115F4890F85E0004281ED0A4F84410D5
:102F4000564890F87000012822D031E043F21E501C
:102F5000A4F8140143F2333014E0387842F6CC423E
:102F6000C0F38100012806D0022804D043F2EB1000
:102F7000A4F8140101E0A4F81421A4F84430DFE718
:102F8000A4F81401A4F84400DAE7A4F81401D0E787
:102F9000387842F26662C0F3810001280FD002281F
:102FA00010D041F6E12000BFA4F81401A4F8442099
:102FB0009BF80020D20708D0BBF8022007E0A4F855
:102FC0001421F3E74FF40050EEE733488288A9F864
:102FD000122010B2B4F944205043C0F38F3250464F
:102FE000AAF812208A4200D9418232490978C906DA
:102FF00005D5428A41F233318A4200D24182218989
:10300000C1F3C002C1F300218A4205D1428A40F6D1
:10301000CC418A4200D94182B17AC90700D04582A9
:10302000BAF81200A06200287FF7EDAE22480570C2
:10303000022099F81A1099B902283FD080B1184996
:103040000B789C0608D5B479640605D5194C24780C
:10305000E40964F386130B70F18821F40261F180B6
:103060000F49496C4E2907DBB179090604D50A4995
:103070000B7823F002030B7089F81A0088F80F0010
:1030800053E600006C0900202C0700202E070020CA
:10309000AC020020600A0020E2050020C00C0020E5
:1030A00048010020100C0140E8050020D004002059
:1030B000640000200407002040070020398F002909
:1030C000BDD143F698213987B9E770B500230C8844
:1030D00063F30F02012505FA03F6344206D0C3F16B
:1030E0000F0605FA06F1114361F30F025B1C102B6A
:1030F000F1DB028070BD70B500230C7863F307022A
:10310000012505FA03F6344206D0C3F1070605FA95
:1031100006F1114361F307025B1C082BF1DB02701F
:1031200070BD0000F0B51F4890F866301E48012BB6
:10313000816821F4006232D11C4BDE8874062ED4E3
:103140001B4D0F054FF00004B5F902501ED4194A6B
:10315000526C642A11DC40F6386295420DDAB204F2
:103160000BD4027852070ED4B0F8D42040F6B8350C
:10317000AA4203D2521CA0F8D420F0BD41F4006151
:1031800081605C81F0BDA0F8D440F0BD41F2CD017A
:103190008D42FADD997AC907F7D18260F3E7826040
:1031A000F0BD0000C00C0020AC020020600A00202E
:1031B000E2050020480100200C490D484B88426C74
:1031C00003B982645B1C9BB24B80FA2B0CD3836CDB
:1031D000D21AC2640020488040F6B830824203DB35
:1031E0000449012081F80D01704700006C0900209E
:1031F00048010020AC020020F0B5364D364F0446A1
:1032000095F83B0097F83B1023780843EE1C627852
:10321000834205D1E0781146FEF776FF207908E079
:1032200094F802C084450CD1E1781046FEF76CFF9B
:10323000E07905F82F0F2878805D6870287BE877A3
:10324000F0BD82421DD161461846FEF75DFF95F83C
:103250004E1095F83B00814207D1B97A09B1A179A6
:1032600000E0617985F82F101EE06978012901D00E
:10327000A17922E0617927E0297841F004012970E1
:1032800012E0E1788142DBD119466046FEF73CFF4F
:1032900095F84E1095F83B0081420AD1B97A09B1F0
:1032A000617ADFE7217ADDE715F82F1F895D697004
:1032B000C5E76978012906D0617A85F82F10B97AB7
:1032C0000029F1D1D8E7217A85F82F10B97A0029A1
:1032D000EAD0D1E758040020480100200B480178CB
:1032E00021F0020100F8381B002100F8181941777D
:1032F000817733218185418508214184012100F8AE
:103300001F1C034880F83910704700005804002043
:10331000480100200D4900B50B4851F8012F40F835
:10332000032F89888180084801210930FEF7FCFFBE
:10333000054802211330FEF7F7FF034804211D3032
:103340005DF804EBFEF7F0BF5804002048010020B0
:10335000094944F648000880091D46F648000880DF
:10336000091D41F2111008800348001F018841F037
:103370002001018070470000182C01402DE9F04722
:10338000664C674B0025A0780126654A1033052856
:103390007ED2DFE800F00313113E1100108820F008
:1033A000010010801D805F480580001F0580001F00
:1033B0000580FFF7CDFFA670BDE8F087594941F2BF
:1033C00044401C390880574945F658002439088084
:1033D000091D47F2580008805249202028390880EA
:1033E0000020401CC0B27328FBD3FFF7B1FF4C494B
:1033F00084F85C502C3147F69060088048481430BF
:1034000006801D80108840F0010010800220A0700E
:10341000D2E700215FF0010004EB410204EB40031E
:10342000B2F85020B3F850309A4200D20146401C06
:10343000C0B20628F0D33C48405C84F83900FFF75E
:103440004DFF1D2000F0F3F900F076F8374E3848B4
:103450004FF4807996F83B10012904D002291BD043
:10346000042930D047E040218046FEF709FF87005D
:1034700080214046FEF704FF47EA400749464046A0
:10348000FEF7FEFE074347F0010084F83B0000E032
:103490003DE0224809302CE040218046FEF7F0FE56
:1034A000870080214046FEF7EBFE47EA4007494689
:1034B0004046FEF7E5FE074347F0020084F83B0074
:1034C0001648133015E040218046FEF7D9FE8700EC
:1034D00080214046FEF7D4FE47EA40074946404671
:1034E000FEF7CEFE074347F0040084F83B000B488C
:1034F0001D3002F05FFF94F82F0086F838001D2081
:1035000000F0ABF90420A0700A48057054E7108859
:1035100020F0010010801D80A5704DE758040020A8
:10352000000800403C2C0140408F0008480100206A
:1035300000100140230700202DE9F041344C14F81D
:103540002F0F344DE07240212846FEF799FE860089
:1035500080212846FEF794FE46EA4006AF1539461C
:103560002846FEF78DFE0643207BF1B22F3C8142B8
:1035700015D084F83C0040212846FEF781FE8600E5
:1035800080212846FEF77CFE46EA4006394628465A
:10359000FEF776FE064384F83B60FFF723F81E4DE6
:1035A00095F83B00012827D0022828D0042829D0EC
:1035B000174894F83B102730085C04F8300F14F8D3
:1035C0000109FEF7E9FE04F82F09A87A00B10120ED
:1035D000607001F025FB94F84E0094F83B1088428F
:1035E00006D094F83800062802D2401C84F838002F
:1035F00084F84E10BDE8F0810548093004E0044825
:10360000133001E002481D30BDE8F041FFF7F4BD82
:103610005804002000100140480100202DE9F0412D
:10362000524991F87200AA287ED191F8730055286A
:103630007AD14F4C00200A5C2254401CC0B274283E
:10364000F9D34C4E2069C6F80100A08AA6F80500FF
:10365000D4F81600F060D4F81A003061D4F81E00D7
:103660001234706102F04CFE4349608A888102F096
:1036700061FE207D123CC007307802D040F004008B
:1036800001E020F004003D4930704FF480403C4D93
:10369000886114F8280F85F82000608B6880A08B63
:1036A000A880E08BE880208C2881608C354F688171
:1036B00094F8240087F8D20014F8011C304686F8EC
:1036C0003B100026C0F89C60FFF724FE2E48A18E18
:1036D0000183E18E4183218F818394F84210283C3D
:1036E000012908D0022901D0032909D0297821F025
:1036F0000C01083107E0297821F00C01091D02E0D6
:10370000297841F00C01297094F86E20012162B1F2
:10371000012A01D0022A0BD087F8461094F86430B1
:103720001A4A4BB1518108E014E087F84660F5E78A
:10373000022287F84620F1E7568194F8701001299B
:103740000AD094F86D1051B101290BD04FF480517B
:10375000A0F87610BDE8F08144F21C71F8E74FF450
:103760000051F5E741F25551F2E7000000FC000876
:10377000C00C00204801002064000020580C0020EC
:10378000D0040020AC02002038050020600A002090
:103790007CB50121082000F089FB4FF48070ADF862
:1037A000040010248DF8074001208DF8060001A9BF
:1037B0001548FEF7E7FC0121092000F077FB012105
:1037C0001248FEF731FD0820ADF8000004208DF806
:1037D00003000F4E03258DF8025069463046FEF770
:1037E000D1FC08213046FEF752FDADF800408DF8BF
:1037F00003408DF8025069463046FEF7C3FC1021A5
:103800003046FEF744FD7CBD00140140000230004C
:10381000000C0140FEE7704700F01F0201219140BB
:103820004009800000F1E020C0F88011704700F0EE
:103830001F02012191404009800000F1E020C0F802
:103840008011704700F01F02012191404009800063
:1038500000F1E020C0F80011704700F01F020121C4
:1038600091404009800000F1E020C0F8001170474D
:1038700070B50F23C47801780122F4B1144C246888
:10388000457804F4E064C4F5E064240AC4F1040655
:10389000E3408478B5401C402C4301F1E021230132
:1038A00081F80034007800F01F018A404009800050
:1038B00000F1E020C0F8002170BD01F01F0082403F
:1038C0004809800000F1E020C0F8802170BD0000B0
:1038D0000CED00E00249084302490860704700000F
:1038E0000000FA050CED00E02DE9F05F00261D2038
:1038F000FFF792FF6C4CDFF8B4B1A4F1B800A77EDB
:1039000090F83810DFF8A8E1DFF8A8A100258F4271
:103910007ED0E776A176626A036B5A434FEA12497A
:103920009BF80820120702D51EF8012000E00A4685
:1039300094F812C0BCF1010F09D004EB4206B6F9AD
:1039400002C0C4F828C0B6F90460E6620CE043F691
:10395000FF7CC4E90A5C90F83DC05FEACC7C01D0F2
:1039600012B102E0052A00D1012600EB47074FF013
:10397000804CBF893F04B7FBF3F3E361476BBCFBAB
:10398000F7F7276294F813C0BCF1000F06D0BCF122
:10399000010F05D03B4403EBD3735B10636201E07E
:1039A0003B466762DFF810C14FF6FF7707EA8307EF
:1039B000ACF808709AF8007090F80A8090F83DC052
:1039C000082F08F003070CF0030C05D067450BD156
:1039D000B8F1000F05D008E0674505D0B8F1000F39
:1039E00003D05B42636200E06562C6B1636A002B8C
:1039F00003D006DD228D05E00AE0304B33F81220BB
:103A000000E0A28DA4F86020227822F0200222702B
:103A10009AF80020042A07D0082A05D012E0B4F84A
:103A2000603003EB0902EDE780F8405065629BF8D7
:103A30000800000701D51EF80110204830F81100D9
:103A4000A4F860001E49606A09883E314843B4F812
:103A5000601001EB204006B21D20FFF7F3FE606A04
:103A6000002807D021784FEA81600ADD002804DAB7
:103A7000A08D09E0B4F8600006E0E06AB04208DB1F
:103A80000CE0002802DA208D208208E0A06AB04213
:103A900004DD208241F02000207000E026822575A0
:103AA00065752586BDE8F09F00020020AC0200206D
:103AB0006C98000823070020380A00207E98000830
:103AC0002404004043184FF48042934210DD90429A
:103AD00002DD104600210BE0914202DD002011467C
:103AE00006E08003B0FBF3F000B2C0F5804109B2FC
:103AF00041EA004070470000F0B54FF46A630022CD
:103B0000C3600E24826204820D4D0826456106833F
:103B100043F6FF774283878340F2492E4FEA873C82
:103B2000C0F808E0C0E9082CCB608A620C824D61C5
:103B30000E834A838F83B4208860C1E9082CF0BDCE
:103B400001060100002181620949C1600E21018244
:103B50004FF6BF514161082101834FF44041418339
:103B600043F6FF7181830907016202494162704790
:103B7000638A010000C0FF0F064941F6A260088079
:103B800005480168054A01F4E06111430160BFF393
:103B90004F8FFEE7442C01400CED00E00400FA05D5
:103BA00038B501210D2000F081F94FF4E060ADF847
:103BB000000018248DF8034003258DF80250694653
:103BC0000D48FEF7DFFA4FF46040ADF800008DF8C5
:103BD00003400A4C8DF8025069462046FEF7D2FA9F
:103BE000A014ADF8000048208DF803006946204677
:103BF000FEF7C8FA38BD000000080140000C014083
:103C00002DE9F0410121CE028CB0304600F04EF992
:103C1000DFF86C81404601F07BFC08A801F0A4FEAF
:103C20004FF45860ADF824000024ADF82040202067
:103C3000ADF822000125ADF826408DF8285008A9DE
:103C4000404601F043FE0021404601F096FE4FF64B
:103C5000FF71404601F09BFE01220021404601F029
:103C600027FE0121404601F00FFC04A801F027FCCB
:103C7000ADF81060A802ADF81200ADF81440A22013
:103C8000ADF816002803ADF81800ADF81A40ADF8ED
:103C90001C4004A9404601F001FC6027ADF800700B
:103CA000ADF80440ADF80840ADF80C40ADF8024066
:103CB000ADF80640ADF80A40ADF80E406946404602
:103CC00001F0E6FC6946404601F028FD69464046A1
:103CD00001F06EFDADF8045040F61450ADF80070E0
:103CE000ADF80600ADF80840ADF80C40ADF8025054
:103CF000ADF80A40ADF80E406946404601F09CFD23
:103D00000121404601F0E4FB0821404601F000FD9E
:103D10003146404601F042FD0821404601F086FD53
:103D20003146404601F0BAFD7021404601F0C3FD26
:103D300018208DF82C008DF82D408DF82E408DF830
:103D40002F500BA8FFF794FD0D480C30018841F06F
:103D5000800101800A481430018841F0010101808E
:103D6000001F04800121404601F0BCFB8DF8285063
:103D70000121404601F0C0FB0CB0BDE8F08100001D
:103D8000002C0140704740F21341416008218160DE
:103D90008621C1604FF480410161494241610021A7
:103DA0000162C162704701627047000010B501886E
:103DB0004288891A09B20183B1F5005F02DBA1F5DF
:103DC000804104E011F5005F02DC01F580410183D0
:103DD000B0F9182041685143C1618368846A534334
:103DE000C2681B12624303EB2222036A1A44114485
:103DF00002628A13426241698A4203DB01698A4294
:103E000000DC11468A1AC0E90A21028E4FF40373BE
:103E1000594302EBA13202860B4A1278082A04D1D8
:103E20000A4A936F03EBA1319167B0F93010B1F5F5
:103E3000804F02DDA1F5804103E0002902DA01F59F
:103E40008041018610BD000023070020740A002075
:103E5000034A516821F4404101435160704700001A
:103E600000100240044A0029516901D0014300E0DA
:103E7000814351617047000000100240044A00294C
:103E8000D16901D0014300E08143D1617047000056
:103E900000100240044A0029116901D0014300E0EA
:103EA000814311617047000000100240044A00295C
:103EB000916901D0014300E08143916170470000A6
:103EC00000100240044A0029D16801D0014300E0FB
:103ED0008143D160704700000010024030B5244992
:103EE0004A6812F00C03234A03D0042B01D0082B9C
:103EF00026D002604A680F231F4C03EA1212A35C0B
:103F00000268DA4042604B68072505EA1323E35C48
:103F100022FA03F383604B6805EAD323E35CDA40BB
:103F2000C2604B68032403F4404104EA933303EB7B
:103F30009161114B1B1F595CB2FBF1F1016130BD66
:103F40004A680E4B1A404B68140103F4803303D5C2
:103F5000C2F38342113202E0022404EB924213B115
:103F60004B689B0301D5064B00E0024B5A43C0E768
:103F70000010024000127A000400002000003C08FB
:103F800000093D002DE9F041274CA61540212046AF
:103F9000FEF776F9850080212046FEF771F945EAA3
:103FA000400531462046FEF76BF90543EDB240214E
:103FB0002046FEF765F9870080212046FEF760F96C
:103FC00047EA400731462046FEF75AF90743F8B260
:103FD000A842DBD140212046FEF752F9870080211C
:103FE0002046FEF74DF947EA400731462046FEF7E6
:103FF00047F90743F8B2A842C8D140212046FEF74E
:104000003FF9870080212046FEF73AF947EA40074A
:1040100031462046FEF734F90743F8B2A842B5D13D
:104020002846BDE8F08100000010014010B502688C
:10403000416802FB02F301FB01330D4CA34211D98D
:104040001B0E0E3B0B4C9BB212B234F8133009B26C
:104050005A43594342F38F3241F38F31C0E9022171
:10406000012102E0C0E902210021017410BD00001D
:10407000E10BBF0E908C00082DE9F05FFE48FF4970
:1040800002880B889A1A92B20F2A7DD30988FC4FB6
:10409000018043F23332B7F91810FA48FA4E00257E
:1040A000DFF8E8A3FA4C914213DBDAF8442040F63B
:1040B000B8318A420DDC94F80D1151B1C18841F03C
:1040C0008001C180F3490A7822F002020A70E57388
:1040D000357081894A0703D48A0701D4CA0703D0FF
:1040E000C28842F4007202E0C28822F40072C280E8
:1040F0008146080702D44846C90604D5B9F8061017
:1041000041F0010102E0C18821F00101A9F8061087
:10411000DC48FDF767FEE048B0F93A00B0F5804FA3
:1041200002DADD49401C02E0DB494FF48040488759
:10413000DAF8501041F6CC40814203DDA06820F04F
:104140001000A060D548028822B1521E0280E5739B
:10415000357029E0B9F8060043041DD4B9F80C20E5
:10416000D30619D4120717D4020615D4820613D425
:10417000020511D4420603D5C94A127812060BD59E
:10418000420709D4C20500E00EE105D4020703D4BA
:10419000820401D4C00607D5C248E573C24A35700F
:1041A000C583158080F82A50E08FDFF800C3A3464E
:1041B00050B1401EABF83E00B648037823F002032E
:1041C00003708BF80F500BE0B248027842F0020205
:1041D00002703078012804D19CF80000062800D134
:1041E00035703078DFF8C8E24FF001080A2876D23F
:1041F000DFE800F0FBDA05DAFAF9DA75F8F702F031
:1042000095F99BF80D015C4608B9FEF7D5FFDFF87C
:10421000809240F62822A9F12C09B9F81610491C01
:1042200089B2A9F81610DAF84400904202DAA9F827
:10423000165015E0984A40F6CC43D2689A420FDBFC
:10424000944A43F69913B2F904209A4208DBB1F577
:10425000FA7F05D3397819B9A9F8165087F8008084
:10426000944A118869B199F805305B1CDBB289F872
:104270000530022B05D3904989F805500B885B1C4B
:104280000B80E17B092912D002297CD0A4F830519F
:10429000B4F84010AB46C9B141F288355946A9F887
:1042A00016B0A84220DA3878012819D01CE07248EC
:1042B0004430FEF7D1F8FDF70FFEDAF84410C9F8E4
:1042C000281041F27C51C9F8181082E2B88A208681
:1042D000F86A7863B86A3863A4F8408036E0C5E1CC
:1042E0007548397001801180744890F8682040F654
:1042F0003A20012A0DD0C4F8D81084F8EA10C9F881
:104300002010B4F9301001F21D52824218D8102347
:1043100017E094F8282102B96949C4F8D81084F844
:10432000EA80B4F9301001F21D528242B4F8D8008C
:1043300000B202D810231A4605E02023022202E030
:1043400020231022002000F0C9FB20865B484FF498
:10435000927390F868105B48012915D0DAF8441080
:1043600040F2DC52914203DAB7F90A209A4215DB97
:10437000B4F8402040F6C413521C92B2A4F8402076
:104380009A420BD212E01AE0DAF8442040F2DC51F3
:104390008A4209DAB7F90A10994205DA86F800B0BC
:1043A00084F8EAB0A0F81AB0BDE8F09F3A4AD268A3
:1043B000002AF9DC42F6E0629142EFDAF4E7BAF85B
:1043C000B620A2F16401B1F5967F02D899F80230C7
:1043D00063B1B2F5C87F17D999F80220012A0CD031
:1043E00012E0D7E0B5E0FCE0F7E0FFE0364989F8FD
:1043F00002800A8822F4805205E0334989F802508D
:104400000A8842F480520A80B4F8302140F6B8316C
:104410008A4207D2184B1C3B1B78DB0702D1521C87
:10442000A4F8302193B240F2DC52934202D842F613
:10443000CC4103E0A4F8301143F26661F967C9F892
:10444000280089F80880214FA4F8405084F8EA50E9
:10445000797F4E4679B1F87FD0B3208DB4F9301012
:1044600000B20A23052200F039FB2086FD777D7714
:10447000B4F916012DE037E06C0900202C0700206C
:1044800064000020600A002023070020480100206B
:10449000AC020020E2050020380500203007002093
:1044A00004070020FC0800201E0000202407002034
:1044B000680200202000002022000020C00C002004
:1044C0009AF9FFFFE0090020442C0140880C0020ED
:1044D00026E0B4F91411884228DAF34991F84D1016
:1044E00011B300F1020023E000B2F04901F0CEFC6C
:1044F000A4F8E400A16A814200DA0846EA4900B261
:10450000B08291F84D100029B4F9301002D0362352
:10451000052202E040F24713362200F0DFFA01E004
:1045200040F266602086A3E7083001E003DD801ECC
:10453000A4F8160101E0A4F81611B4F930004FF404
:104540008041884201DD21862EE70028FCDA25869D
:104550002AE7D74ADBF8DC105846914202D2491CC0
:10456000C0F8DC10C17B082903D1D0F8DC109142DF
:104570000CD335708168CA0502D521F0080101E02D
:1045800041F008018160CBF8DC500DE7BDE8F05F39
:1045900002F0FEBC9BF80F005F46092803D03D8661
:1045A0008BF80F5054E1C34CE069401CE0610228D5
:1045B00009DD208D012301B2208B052200B200F01D
:1045C0008DFAE561A062BC48218D0180BAF84410E3
:1045D0004180FDF759FF3886E6E6BDE8F05F04F05C
:1045E00019BA9EF8000009287ED0DDE6B14AB3482A
:1045F0009570038843F4805303808BF80D519BF82A
:10460000283163B141F31100CBF8D850AC49830392
:10461000F86280108B628103B862AA488162D582F9
:10462000DAF8441041F28830814207DA38780128FC
:1046300004D1A5483D700580A4480580A44AA54B37
:104640001088401C81B2A4481180C82902D3047884
:10465000012C17D0B1F57A7F02D30478022C11D047
:10466000B1F5FA6F02D3017803290BD09BF80F0044
:10467000801E082875D2DFE800F010AEEDFD04744E
:1046800075A091E605701580B9F8061021F4006157
:10469000A9F8061083F80080E8E7FDF72BFE9AF8EA
:1046A00000005446400612D58C48807804280ED06D
:1046B000616C204682290ADA817A94F83D0001F083
:1046C000030100F00300814201D001F0DFFD3078EA
:1046D00006288AD084F83F50206DA94640F3110087
:1046E00082037749F86200E0B2E080108A628103B9
:1046F000B86274488162FDF7EFFB6E485D4680F852
:104700000880BBF81401ABF81601606CABF882901E
:10471000B0F5437F12DD4FF48040A5F88000A86813
:1047200040F48060A86094F838100529A9D140F0C1
:104730001000CBF8080089E0307035E64FF4804176
:10474000A5F88010A96821F48061A96040F28A214F
:10475000884204DA2078400601D402F005FBA868FC
:1047600071E098E0DAF84400B0F5437F07DA9CF88E
:104770000010062903D000BF8CF8005083E0584891
:10478000017821F040010170FDF7A6FB43F6FE70B1
:10479000ABF816010BF1DC04FDF7ACFD514810F845
:1047A000341F21F001010170464925608D624449A2
:1047B0008D62082131704564F6E53F48FDF74CFEF7
:1047C000FDF78AFB3B48DAF84410816241F27C51E4
:1047D00081610920B0E799F80600C006ADD4DAF887
:1047E00044005446B0F57A7F32DDFDF783FD207832
:1047F000400611D53948807804280DD0606C822895
:104800000ADAA07A94F83D1000F0030001F00301E9
:10481000884201D001F03AFD84F83F50B4F85000CE
:10482000ABF8300001B24FF480405D46814200DDBC
:104830002886FDF751FBA86840F48060A86094F8D2
:1048400038100529B8D140F01000A860022073E7A5
:104850003570A9E5DAF84400B0F5437F03DA9CF837
:104860000010062988D1B9F8061021F02001A9F816
:10487000061000E003E0FDF73DFD04205CE79CF836
:104880000000062802D086F800808DE509208EF809
:104890000000052050E7114885708CF8005087F81B
:1048A0005E50ABF830507FE5C00C0020828E0008CF
:1048B000C0D4010080020020B0090020442C014037
:1048C000CC0800209C0800202200002020000020AE
:1048D00016000020140000201500002058040020BD
:1048E00032070020740A002030B585B00121042071
:1048F000FFF7DCFA4FF40040ADF8100048208DF8C7
:10490000130004A91848FDF73DFC01210846FFF7F4
:10491000B5FA40F68C20ADF8040003240020ADF871
:104920000040ADF80200ADF806004FF08045694642
:10493000284600F0CBFF1C208DF80C008DF80D40B0
:104940008DF80E4001208DF80F0003A8FEF790FFB0
:1049500001221146284600F093FE0121284600F06E
:10496000C1FD05B030BD00000008014070470000E7
:104970002DE9F041304CE07800285AD12078002809
:1049800057D0401E10F0FF00207052D14FF49670A7
:10499000208272B6294F45F2AA50A7F87200002073
:1049A000FDF778FA264D13202860FDF785FAA8BB9D
:1049B0003420E86002202861224E6E61286940F0B0
:1049C00040002861FDF778FA40BB00211E4A0846E6
:1049D0005FEA255312F800C0BCF1FF0F00D001219F
:1049E000401C80B29842F5D3C1B9C4E90676392695
:1049F0000127A06910F8011B10F8012BA061E069E4
:104A000001EB022102886A612F6120F8021BE0613C
:104A1000FDF752FA10B9761EB6B2EAD20120FDF7C0
:104A200039FA62B601F086FC0848816821F48041B9
:104A30008160BDE8F081000020070020C00C00204C
:104A40000020024000FC000800FC0008AC0200202E
:104A50001948016841F010010160016821F003016B
:104A60000160016841F00201016014484168416041
:104A700041684160416841F480614160416821F4CE
:104A80007C11416041680E4A11434160016841F068
:104A90008071016001688901FCD5416821F0030142
:104AA0004160416841F0020141604168C1F3810108
:104AB0000229FAD170470000002002400010024095
:104AC0000000280830B5044C039D6080A180E2807E
:104AD0002381658130BD0000540A00200A448242CF
:104AE00001DA10B27047C91A8142FBDD08B2704783
:104AF0002DE9F0434348DFF81081DFF81091C17FC2
:104B0000457A046801260023414A424880292BD374
:104B100001F01F0158F821100C420146096802D02B
:104B200041F4805101E021F480510160CF0417D499
:104B30008F0415D5977AFF0707D0538199F800C0E5
:104B40002CF0020C89F800C00AE090F84670BFB162
:104B50004FF0020C012F18D080F8463080F81AC1AF
:104B60000F0B67F34D310160802D2AD305F01F0133
:104B700058F821100C4201680CD041F004010BE000
:104B800080F8466080F81A31EAE780F846C080F87D
:104B90001A61E5E721F0040101604C070DD44C05D2
:104BA0000BD5947AE40708D0538199F8005025F08A
:104BB000020589F80050C0F898308C0864F38A2107
:104BC0000160917AC90717D1134991F8641001293E
:104BD00012D11249496C32290CDC0178490709D5F8
:104BE0000189090506D4D0F8981047F23054A14243
:104BF00004D95681C0F89830BDE8F083491CC0F84C
:104C00009810F9E7E8050020A8930008E2050020C5
:104C1000600A0020AC020020C00C002048010020E7
:104C200010B5FCF79FF80F48018821F002010180C0
:104C30000C49183109880C4A928E1144094A3432C1
:104C4000118008490C390A8842F001020A80011DCE
:104C50000A884FF6ED531A400A80018841F012018C
:104C6000018010BD0C040040580400200648418813
:104C7000491C89B24180B1F57A7F04D38188491CEF
:104C80008180002141807047440700200F4810B503
:104C9000016841F00101016041680D4A1140416025
:104CA00001680C4A11400160016821F48021016013
:104CB000416821F4FE0141604FF41F018160FFF75C
:104CC000C7FE05494FF00060086010BD00100240AB
:104CD0000000FFF8FFFFF6FE08ED00E02DE9F041CF
:104CE0003149324D0888401C088028884FF0000464
:104CF000000629D5FCF7B6F92D4A2E480723177868
:104D0000C8262D49012F22D02C4FB7F806C0BCF180
:104D1000000F3ED0B0F80CC04CF0080CA0F80CC04E
:104D2000B0F806C02CF4006CA0F806C0886820F02B
:104D300004008860FC801370CE8700204FF49661D9
:104D4000401C80B28842FBD32C80BDE8F0811C4F10
:104D500097F800C0BCF1010F0FD0BCF1020F11D0C9
:104D6000B0F806C04CF4006CA0F806C0886840F0AB
:104D70000400886005203870DDE7B0F80CC04CF006
:104D8000080C03E0B0F80CC04CF0100CA0F80CC0FC
:104D9000F0E70C4F3C70C78847F40067C78088680D
:104DA00040F004008860C6E744070020102C014052
:104DB00023070020600A0020AC0200206C090020BC
:104DC0002407002041070020704700002DE9F04330
:104DD0004FF08040018A21F001010182AC48007847
:104DE00000287CD1AB4FF87B002878D1AA48406CD2
:104DF000322874DCA9488068DFF8A4924104A94DE8
:104E0000B9F804004FF0000403D4401CA9F80400D2
:104E100028E1002874D02978012611B1012912D087
:104E200017E14946B0F5BE7FFAD92E70CC718C716E
:104E3000EC702C72287A0A18401CC0B214722872C6
:104E40000F28F7D305E1B9F802204946824201D97B
:104E5000EE7100E0EC7192488A7908300F2A15D281
:104E6000CB79082B0BD2C3F10708EB7912F800C0FD
:104E700003FA08F363441354CA79521CCA71CA79FD
:104E8000082A03D18A79521C8A71CC7199F80610CC
:104E9000C8460F2973D10D21FCF74EF8A881010AED
:104EA0006970C0B2A87088F8064098F816208A4247
:104EB00065D198F81510814261D198F80BC07A49F4
:104EC000032302227948BCF1000F10D0BCF1010F7E
:104ED00002D0BCF1020F14D080F86A2000E0CBE0D1
:104EE00091F800C02CF00C0C0CF1080C0FE080F8CD
:104EF0006A6091F800C02CF00C0C0CF1040C06E078
:104F0000A9E080F86A3091F800C04CF00C0C81F8F0
:104F100000C098F80C10B6EB111F04D180F86E4059
:104F200087F846400EE0B2EB111F04D180F86E60A6
:104F300087F8466006E0B3EB111F03D180F86E20BE
:104F400087F846200B0717D001F00F01012901D087
:104F5000022915D080F86C602C7198F80D102A7910
:104F600006FA02F30B406B71082A44D2DFE802F024
:104F70000B124319242F363D80F86C40ECE768E0B3
:104F800080F86C20E8E713B180F8704033E080F8D7
:104F9000706030E013B180F850602CE080F8504031
:104FA00029E023B180F8656087F8036123E080F889
:104FB000654087F803411EE023B187F8F54080F88B
:104FC0004D4018E087F8F56080F84D6013E013B1AC
:104FD00080F868600FE080F868400CE013B180F85A
:104FE000666008E080F8664005E013B180F867600D
:104FF00001E080F86740521CD2B22A71082AAED371
:1050000098F80E102A4A8B0705D587F8F16080F8CA
:105010006460568104E087F8F14080F86440548170
:10502000C90702D080F8294001E080F8296098F88B
:10503000111000F86D1FC2781E48012A1ED001B35E
:10504000012921D04FF48051A0F876101A493C2054
:105050000870A9F80240A9F80440B9F80210491CE8
:10506000A9F80210B9F80210B1F5FA7F04D940F29C
:10507000F511A9F802102C70BDE8F08344F21C7100
:10508000E2E74FF40051DFE741F25551DCE7000061
:1050900023070020AC02002048010020001001403E
:1050A000A80C0020BC060020D0040020C00C00206A
:1050B000600A002038050020200700202DE9F05F5D
:1050C000FDF718F98E4D2888A5F10406C0070AD00F
:1050D000308820F008003080288820F009002880DF
:1050E00001F042FED9E02888DFF81892DFF8188234
:1050F000864C80071AD5B9F8001041F00101A9F8D3
:105100000010B8F800008049143150300880288819
:105110004FF6F95108402880308840F00400308074
:10512000FEF730FF84F83C00BDE8F09F2888784FF8
:105130004007288871D520F004002880FEF722FF60
:1051400094F83C108142EFD1308820F00400308088
:10515000FDF7A8FA2078410605D594F8541094F884
:105160003B209142E0D03978400621F002013970AD
:1051700004D5FEF7E1F997F82F7004E094F83C00AD
:10518000FDF70AF90746DFF880B140F68C2A0BF1EB
:10519000180B062F47D294F83800B8423ED0384654
:1051A000FDF77EF82078C00716D094F83A0094F8FE
:1051B000391000F00302914206D0A17A00F00100FC
:1051C00001F00101884215D1FDF7D4F9FBF716FE75
:1051D000FDF7FCFA384689E0FDF7CCF9FBF70EFE47
:1051E000FDF7F4FA3846FDF7E5F9207840F00100C4
:1051F000207099E7288820F008002880206B81081B
:1052000001EBD000504515D2B8F800100844ABF8B7
:105210000000308840F0080003E00DE0308820F006
:105220000800308080E7B9F8001041F00101A9F8CA
:105230000010DFE75046E7E70007288831D520F067
:1052400008002880308820F008003080FEF79AFEA1
:1052500084F83C00FDF726FA387820F00200387018
:105260002078400604D5FEF767F997F82F5004E040
:1052700094F83C00FDF790F80546062D08D294F806
:105280003800A842B5D0FDF775F9FBF7B7FD2AE065
:105290002048C18841F04001C180BDE8F05FFDF7C2
:1052A00075BAC006288825D520F0100028803088DF
:1052B00020F01000308097F838000C2802D2401CF3
:1052C00087F83800387840F002003870FEF734F97B
:1052D00097F82F50787884F8390094F83800A8426D
:1052E00087D0FDF747F9FDF771FA2846BDE8F05F72
:1052F000FDF760B94EF2BE110840288014E70000A7
:105300001004004000040040240400404801002034
:1053100058040020600A00202DE9F04F514F85B05D
:10532000388820F0010038804E4800261030068072
:105330004D4CDFF838A14FF0010894F85C0042F6BC
:105340003029C10774D072B64948816941F40071AF
:105350008161816941F4806181614FF40040FEF711
:1053600077FD444D00212846FBF7A6FA0021284688
:10537000FBF798FADFF800B100215846FBF792FAE4
:1053800000213E48FCF702F92846FBF7B1FB5846DE
:10539000FBF7AEFB4FF46020CDE902068DF8056007
:1053A00000968DF810808DF8048069462846FBF73A
:1053B00031FC01231A460F212846FBF77CFC012112
:1053C0002846FBF76FFA00204946401C80B288420D
:1053D000FBD328462E600121FBF7ACFC2868800730
:1053E000FCD524484C30006894F85C1021F0010191
:1053F0002144A1F85000FBF769FA62B6FDF7A8FF57
:1054000047F69061AAF8001094F85C00401CC0B206
:1054100084F85C000C2822D212491431A1F80080D3
:10542000388840F00100388005B0BDE8F08FFFE714
:10543000134920F00100085A12490880114945F625
:105440005800083908800F4847F25801001F0180B2
:105450000C4920200C390880AAF80090D4E70320DA
:10546000A070E1E700080040580400202C0800402C
:1054700000100240002401400028014008000240C2
:10548000648F0008202C01400029018802D041F0DF
:10549000800101E021F080010180704710B50A8889
:1054A0004B88CC881A438B8823431A430B891A43B1
:1054B0004B8989891A430A43A0F8442010BD002172
:1054C000018041808180C18001814181818170475B
:1054D0000029818802D041F0010101E021F00101A1
:1054E000818070470029018802D041F0010101E06C
:1054F00021F0010101807047002930F8441F02D0DB
:1055000041F4004101E0C1F30E0101807047000049
:105510004B4910B5884202D10121C41486E0B0F194
:10552000804F09D0474988420DD101210220FEF762
:10553000B1FC0021022064E001210846FEF7AAFC2C
:10554000002101205DE04049884206D1012104206C
:10555000FEF7A0FC0021042053E03C49884206D11C
:1055600001210820FEF796FC0021082049E0384977
:10557000884206D101211020FEF78CFC002110206A
:105580003FE03449884206D101212020FEF782FC09
:105590000021202035E03049884202D10121441405
:1055A00044E02E49884202D10121CC043EE02C493E
:1055B000884202D101210C0538E02A49884202D1F3
:1055C00001214C0532E02849884206D101214020C2
:1055D000FEF760FC0021402013E02449884206D1F8
:1055E00001218020FEF756FC0021802009E020499F
:1055F00088420AD1841501212046FEF74BFC002188
:105600002046BDE81040FEF745BC1A49884202D149
:1056100001210C040AE01849884202D101214C04FE
:1056200004E0164988420AD101218C042046FEF785
:1056300049FC2046BDE810400021FEF743BC10BDE8
:10564000002C01400004004000080040000C004015
:10565000001000400014004000340140004C0140A4
:10566000005001400054014000180040001C004060
:10567000002000400040014000440140004801403B
:10568000002A828901D00A4300E08A438281704760
:1056900030B5028C22F001020284028C8388048BD4
:1056A00022F0020224F073050C882C430D89154367
:1056B0004A882A43114DA8420BD0114DA84208D068
:1056C000104DA84205D0104DA84202D00F4DA8425F
:1056D0000DD122F008054A8923F440732A4322F0B1
:1056E00004058A882A438D891D43CB892B438380F7
:1056F0000483C9888186028430BD0000002C0140EB
:105700000034014000400140004401400048014095
:10571000028B22F008020A430283704770B5028CA4
:1057200022F010020284028C8488038B0D8823F4FB
:10573000E6464FF6FF7303EA052535430E8922F04E
:10574000200203EA061616434A8803EA021232438D
:10575000104EB04202D0104EB04215D122F0800659
:105760004A8924F4406403EA0212324322F04006DC
:105770008A8803EA021232438E8903EA86062643A8
:10578000CC8903EA8404344384800583C988018773
:10579000028470BD002C014000340140028B4FF6A2
:1057A000FF7322F4006203EA012111430183704771
:1057B00070B5028C22F480720284028C8488838B00
:1057C0000D8823F073031D4322F400730E894FF6F6
:1057D000FF7202EA06261E434B8802EA0323334384
:1057E000104EB04202D0104EB04215D123F40066E4
:1057F0004B8924F4405402EA0323334323F48066A4
:105800008B8802EA032333438E8902EA0616264375
:10581000CC8902EA0414344384808583C988818753
:10582000038470BD002C014000340140828B22F0C3
:1058300008020A438283704770B5028C22F48052BA
:105840000284048C8288838B0D8823F4E6464FF60D
:10585000FF7303EA0525354324F400560C8903EA57
:10586000043434434E8803EA06362643094CA042EA
:1058700002D0094CA04205D122F480448A8903EA6F
:105880008212224382808583C988A0F84010068452
:1058900070BD0000002C014000340140828B4FF6A7
:1058A000FF7322F4006203EA0121114381837047F0
:1058B000018582827047828822F07002828082880D
:1058C0000A4382807047A0F84010704730B50288C4
:1058D0001B4B1C4C98420DD0A0420BD0B0F1804F16
:1058E00008D0194DA84205D0184DA84202D0184D35
:1058F000A84203D122F070054A882A43154DA842D8
:1059000006D0154DA84203D022F44075CA882A4318
:1059100002808A8882850A88028598420AD0A0423D
:1059200008D00E4A904205D00D4A904202D00D4A4E
:10593000904201D1097A01860121818230BD0000A7
:10594000002C0140003401400004004000080040E9
:10595000000C0040001000400014004000400140D6
:1059600000440140004801404FF6FF718180002152
:105970000180C1804180017270470029018802D0F6
:1059800041F0020101E021F002010180704700298D
:10599000018802D041F0040101E021F004010180FE
:1059A0007047000030B52348244B90F8201002685F
:1059B00001F01F00204951F820000242186802D06F
:1059C00040F4803001E020F4803018601C484FF033
:1059D0000005807941061B482AD41B4902880C889F
:1059E000A21A92B201240F2A12D30A880280826876
:1059F000002A00DA5242062A0ADD144A1278022AE4
:105A000006D193F80D2102B94477C5770A88428000
:105A1000427F012A02D00988418030BD428809882E
:105A2000891A89B240F21A629142F6D3C47730BD26
:105A3000457730BDE8050020A8930008AC0200209F
:105A4000600A0020880C00202C070020230700207B
:105A50002DE9F0414D6800231E240F22854202DD0E
:105A60000868BDE8F081D1F8F450854202DAD1F837
:105A7000F000F6E701EBC2056D68854201DA1346D6
:105A800000E01446E21852085D1CAA42F2D101EB74
:105A9000C20351F832505C68844202DAD3E90267EB
:105AA00001E053E90267001BC11789053A1B41EA6F
:105AB0009021D3178005FAF735FB721BA0FB024635
:105AC00001FB0261D31700FB0310810241EA9450ED
:105AD0002844C6E72DE9F04FDFF8B8B16A48DFF88F
:105AE000AC91DFF8ACA190F80EC0BBF91A70BBF90D
:105AF0001C60BBF91850BBF96C10BCF1070F48D201
:105B0000DFE80CF08D041A30485E7600D9F80020EA
:105B10008284DAF80020C284828CC38CA7EB8202D4
:105B200012B2A6EB83034A431BB2594342F3CF227E
:105B300041F3CF23D11870E0D9F800204284DAF87D
:105B40000020C284428CA5EB820213B2C28C4B436C
:105B5000A6EB820212B243F3CF24514341F3CF2389
:105B6000E11814E0D9F80020C284DAF80020428459
:105B7000C28C438CA6EB820212B2A5EB83031CB24B
:105B80004A43614342F3CF2341F3CF2419194942D9
:105B90000AB244E0D9F800208284DAF80020428476
:105BA000828C438CA7EB820212B2A5EB83034A439B
:105BB0001BB2594342F3CF2241F3CF24111914E011
:105BC000D9F800204284DAF800208284428C838C49
:105BD000A5EB820212B2A7EB83034A431BB242F346
:105BE000CF24594341F3CF22A11849420BB216E00A
:105BF000D9F80020C284DAF800208284C28C838C19
:105C0000A6EB820212B2A7EB83031CB24A4342F313
:105C1000CF23614341F3CF22991849420CB2BBF91B
:105C20001E50594605F21E56A64201DACE8306E002
:105C3000A5F21E55A54201DDCD8300E0CC83B1F96C
:105C4000204004F21E55954201DA0D8406E0A4F2CC
:105C50001E54944201DD0C8400E00A84B1F9222034
:105C600002F21E549C4202DAABF8224008E0A2F293
:105C70001E529A4202DDABF8222001E0ABF822303E
:105C8000417B8173BDE8F08FAC0200203C240140D1
:105C90003C280140380500202DE9F04704466D48B6
:105CA0006E4E002702786C48022AB0F9301004D0FA
:105CB000082A7BD0092A7AD0C8E0C27B022A02D106
:105CC000B0F8402052B1A4F8421071810423B6F913
:105CD00008101A460020FEF701FFAEE06049DFF829
:105CE0008481496A0D14E5808068410216D5B4F9B3
:105CF000020040F2DA21884248DD40F26A418842DF
:105D000005DD00BF0823B4F942101A4660E0A0F296
:105D1000DA20FAF782FB0022534B68E0C0F3C0019F
:105D2000C0F30020DFF8449181420CD1D8F8440040
:105D300040F2BA4188426DDD40F66A118842E1DCEA
:105D4000A0F2BA404FE04A480078C0060CD5D8F817
:105D5000440041F2243188425CDD41F2D471884232
:105D6000D0DC00F6DC401EE04248DFF80C9190F8F1
:105D7000701001290BD090F86F00012807D03F4820
:105D80000178C90746D03E49098889B142E0B4F993
:105D9000020041F6DC6188423CDD42F23411884267
:105DA00012DC00F59270A0F500501CE047E04BE0DB
:105DB000B0F91000B4F90210A0F59672914229DDF5
:105DC00000F5967291420BDDB4F9421020231A4679
:105DD0000020FEF783FEA4F84200002817DB1BE03A
:105DE000081A00F59670FAF718FB00224B46FAF7EE
:105DF00080FA0E22FAF7ECFAFAF746FB00B2C0F589
:105E0000804068438013A4F84200002D04DCA4F80D
:105E1000427001E0A4F84250B4F842101948F180F1
:105E2000D8F844304364A0F84C10B0F84E1071819B
:105E300098F80A10008F01B94042308106E01248FC
:105E4000B0F87C00708100E07181378184F8407087
:105E5000BDE8F08723070020AC020020640000208A
:105E600038050020480100200000794000C0924021
:105E700004070020C00C002000C082405009002010
:105E800020000020FC080020740A00202DE9F041C9
:105E9000B1F9025000232B241522854203DAB1F90F
:105EA0000000BDE8F081B1F9AE50854202DDB1F9E4
:105EB000AC00F6E701EB8205B5F90250854201DD41
:105EC000134600E01446E21852085D1CAA42F1D1C4
:105ED00001EB8205B5F90230834206DA35F9026C2E
:105EE00035F9044C31F9221006E01E4631F9224002
:105EF000B5F90630B5F90410801B091BC5178911C7
:105F0000AD0345EA90458703A1FB070CCA1702FBC6
:105F100007C201FB05219A1BD317FAF703F9000A00
:105F200040EA0160001900B2B0F5804FB9DB43F6DA
:105F3000FF70B6E770B5134C40F224452946204661
:105F400000F03EF800281BD0204600F0C7F8294694
:105F5000204600F01DF80C4C00212046FBF716FBF4
:105F60002046FBF791FBC0F164000849C0B2042849
:105F7000087201D900F046F9BDE87040FBF7CABBD2
:105F800070BD000000380140580002407406002037
:105F90000A0A01219140C943018070470029818983
:105FA00002D041F4005101E021F400518181704799
:105FB000002A828A01D00A4300E08A438282704725
:105FC00030B501F01F0201240025C1F3421304FA89
:105FD00002F2012B0FD0022B0FD0838A4FEA11213E
:105FE0000088134204FA01F400EA040001D000B171
:105FF0000125284630BD8389F0E7038AEEE710B516
:10600000C1F3421301F01F040121A140012B07D06D
:10601000022B07D01430002A026805D00A4304E09E
:106020000C30F8E71030F6E78A43026010BD00003C
:1060300030B50446008A85B00D464CF6FF71084025
:10604000E98801432182A1894EF6F3100140A88816
:106050002A8910436A890A431043A081A08A4FF617
:10606000FF410840A9890143A1826846FDF736FF38
:106070001948844201D1039800E00298A1890904DB
:1060800000EBC00101EB0010296801D5490000E0D8
:106090008900B0FBF1F06422B0FBF2F109010B09B9
:1060A0006FF018056B4300EB8300A3891D044FF0CC
:1060B000320306D503EBC000B0FBF2F000F007009E
:1060C00005E003EB0010B0FBF2F000F00F00084316
:1060D000208105B030BD0000003801408088C0F349
:1060E00008007047F8B501210920FDF7DFFE012106
:1060F0008803FDF7DBFE10258DF803502020ADF856
:1061000000001A4E03248DF8024069463046FCF721
:1061100039F816490C31086820F020000860182072
:106120008DF803004020ADF800008DF8024069466C
:106130003046FCF727F848208DF803008020ADF8A2
:10614000000069463046FCF71DF88DF80350280121
:10615000ADF800008DF8024069463046FCF712F8B1
:1061600001210420FCF760F8F8BD0000000C01409C
:1061700030B585B0FFF7B6FF00244FF4E130009052
:10618000ADF808400C201D4DADF80440ADF80A00F4
:10619000ADF80640ADF80C4069462846FFF748FFC9
:1061A00025208DF8100004208DF811008DF8124084
:1061B00001208DF8130004A8FDF75AFB012240F2DC
:1061C00024412846FFF71BFF01212846FFF7E6FE82
:1061D000FBF7CAFA012280212846FFF7E9FE0122D7
:1061E00040212846FFF7E4FE012202210448FBF784
:1061F0005FFAFBF7B9FA05B030BD00000038014086
:106200004400024070B51D4D00242878432834D145
:106210006878462831D1A878502807D0512805D071
:10622000812803D0892801D0212826D1144E7071ED
:10623000E9787172A81C891CFAF7B6FEB072717AFF
:10624000294409793182884217D106F10E0001787C
:1062500041F0020101700B48016841F0200101602A
:10626000317A0948002204E02B5D03552A55641C4D
:10627000E4B28C42F8D38078707170BDBC07002006
:10628000740600200C0C0140F20B002070B51D209C
:10629000FDF7CDFAFDF750F91D20FDF7DEFA1548A0
:1062A00090F82F10144D0623144C85F8381090F8F0
:1062B0003B1095F83B201143012A04D0022A07D055
:1062C000042A0AD010E0827A8A420DD0007B09E0CD
:1062D000027D8A4208D0807D04E0827F8A4203D01A
:1062E00090F82000884200D12370002085F84000FB
:1062F00070BD000058040020480100202307002042
:106300000B4800214180A0F1B8018A898280CB89A5
:106310001A44C2800B8A1A4402814B8A1A44428171
:10632000898A1144818143F6FF71C1817047000061
:1063300000020020084940F61C72B1F90C0090429E
:1063400002DA00F59F7005E041F2E302904201DDC0
:10635000A0F59F70C88170476400002038B51348CD
:10636000C16941F00401C1611E208DF800000220C6
:106370008DF801008DF8020001248DF80340684675
:10638000FDF776FA0A4984200880094947F69060AB
:106390002C3108800020091F0880054914310C8029
:1063A000091F0880081F048038BD0000001002404B
:1063B0000008004030B420491E4A45788B7A1146C7
:1063C00092F83B4091F83910AC4218D14BB10379A7
:1063D000994202D04379994201D140791AE08079FB
:1063E00009E08379994202D0C479A14202D182F8AE
:1063F0002F3011E0407982F82F0030BC7047C5780B
:10640000AC42FAD16BB1C379994202D0037A994276
:1064100005D1007A82F82F0030BCFEF701BC407A2B
:10642000E9E7437A9942E2D00479A142DFD0007AC9
:10643000E1E700005804002048010020FEE70000CA
:106440002DE9F0470446007F012868D13548E188EE
:106450000288511A89B2072916D30088E080B4F95E
:10646000000044F2DD414843401346F6D9614843F9
:106470008013A060401000B2A0814FF08051B1FBAA
:10648000F0F0F9F7C5FF2061B4F90C6096B1B4F9EA
:1064900002104DF6B05048430014A082B4F90470C5
:1064A0004DF6B05207FB02F24FEA2245E58204D4D2
:1064B000024603E00020E08330E0424212B2228331
:1064C000002D01DB2B4600E06B421BB2DFF8589039
:1064D000638398464FF4804AB24208DAF9F78FFF97
:1064E0002169F9F762FEF9F7B6FF801304E000298D
:1064F00001DA484600E05046E083B04509DA284614
:10650000F9F77DFF2169F9F750FEF9F7A4FF801331
:1065100004E0002F01DA484600E050462084BDE840
:10652000F08700002C07002000C0FFFF70B53B483B
:106530003B4D3C4C0078022805D1E87B022802D173
:10654000B5F8400028B1288EA4F84E00002020871E
:1065500070BD3448324995F80D21B0F8440091F8E7
:10656000461000B240F6AA262AB119B3012928D054
:10657000022933D03CE0E9B12B490978C1F381010C
:1065800001290CD002290DD02849FBF753FC80B219
:10659000A4F8400095F84610012906D028E02349C8
:1065A000D83909E021496C3906E0B04220D340F6E1
:1065B000F41003E01D496C31FBF73CFCA4F84000EB
:1065C00016E01A49FBF736FC80B240F63E11A4F8FB
:1065D000400088420CD3A4F8401009E01349FBF7AF
:1065E00029FC80B2A4F84000B04201D3A4F8406076
:1065F0000C49B4F840004831383401F083FAB4F95A
:106600001400B4F912204142514389132180B4F996
:10661000101048438013E08270BD00002307002063
:10662000AC020020FC080020D00400208C8D000863
:106630000348002180F82A10C183018770470000B9
:10664000FC08002010B504000B462D4AC3F10000E1
:1066500028D56442002B12DAA04207DA214600F066
:106660002DFA32F81000C0F5404041E001462046C6
:1066700000F024FA32F8100000F5004038E0A342A0
:1066800008DA2146184600F019FA32F8100000F531
:1066900040402DE0204600F011FA32F81000C0F51D
:1066A000803025E0002B12DAA04207DA214600F004
:1066B00005FA32F8100000F5804019E00146204646
:1066C00000F0FCF932F81000C0F5004010E0A342E1
:1066D00008DA2146184600F0F1F932F81000C0F54A
:1066E000804005E053B1204600F0E8F932F8100090
:1066F000B0F5004F01DDA0F5803010BD002010BDC9
:10670000708F000840438013494300EBA130002202
:106710000302002B14DDB3F5001F01DC802001E033
:106720004FF4005093FBF0F1014401EBD17149109B
:10673000814206D0521CD2B20846062AF2D300E0AB
:106740000021C80000B2704702E008C8121F08C14B
:10675000002AFAD170477047002001E001C1121FE2
:10676000002AFBD1704700002DE9F047A74CA8484C
:1067700021880288511A89B20F297DD30088A4F19B
:106780003C052080288F08B1401E288795F800C05E
:10679000A04ACCF3810001281DD0022820D0D18B43
:1067A0009D4E9A48DFF87492F388407E0027B1F539
:1067B000926F1CD8142818D37820607643F010000C
:1067C000F08040F26660A8812CF001002870D77339
:1067D00089F8007018E0D08B00EB4000C00302E0A5
:1067E000D08B8F494843010CDAE7401C04E0B1F537
:1067F000DB6F09D310B1401E607605E023F0100076
:10680000F0804CF001002870B5F90200B5F91430A1
:106810004143C3EBC303C1F38F31C3F3D10303EB94
:10682000510109B2A9829046D28B4FF08053504358
:10683000B5F91620C0F38F30C2EBC202C2F3D10209
:1068400002EB500000B2E882AA6A42431213EA62E5
:1068500093FBF2F22A63734A1080A2680A44A26092
:10686000E1680144E160207C401CC0B2207407282C
:1068700002D942F3CF0000E0C5E02883C910698344
:10688000E760A76041F6C8012774884204DD298BC0
:10689000654AB2FBF1F1E981C117890341EA9041F0
:1068A000800342F69B420023F9F73CFCA88457483A
:1068B0005E49A0F13C002A78B0F906005FEA827CCC
:1068C00000FB01F14FEA2143C2F3810115D50129F3
:1068D00007D002290BD04FF2685141430914A1801F
:1068E00011E049F68C4148430014A08020E04CF6AA
:1068F000183141430914A18026E001290ED0022954
:1069000018D0A0806B844A4948430014A4F81E00A4
:10691000FBF7B0F847480088C0B143E04AF65C3165
:1069200041430914A1804BF62C214843001468848C
:10693000E383EDE74DF2AC5141430914A1804EF2DF
:106940007C414143091469843B49DDE795F8200007
:1069500000BB88F80F7089F80070B5F91A00A0F52F
:106960000C519F39B1F56E7F18D8617FF42912D987
:106970003249E8802E4AA1F8460050430014A8800E
:10698000A1F84400FF2085F8200081F828002C4958
:106990003C20087006E0491C617703E0607F08B185
:1069A000401E6077B5F91A10B4F91E0081420EDD61
:1069B000A07E7D2809D9F08840F00800F0802148A9
:1069C000017821F0020101700EE0401C06E0A0F207
:1069D0003D10814208DAA07E10B1401EA07603E08F
:1069E000F08820F00800F080B5F9181060690844BC
:1069F0006061217E491CC9B221761F2903D940114B
:106A0000A88367612776BDE8F08700000C050020A9
:106A10002C070020AC020020600A00202307002081
:106A200030330100140A002074E8260BCC0E01005C
:106A3000488501002E070020D0450100C00C002031
:106A400020070020E2050020024941F68B308862D1
:106A500070470000D004002070B5164C0625207841
:106A6000062825D2DFE800F003080E141A21124888
:106A7000FAF7D8FA012016E00F48801DFAF7D2FA8B
:106A8000022010E00C480C30FAF7CCFA03200AE0A0
:106A900009481230FAF7C6FA042004E00648183014
:106AA000FAF7C0FA0520207070BDFAF7DBFA2570FE
:106AB000257070BD24070020648E0008090A05D0E7
:106AC000B0FBF1F0FF2800D9FF207047002070478D
:106AD000D0E90021C368521A5A4301EBA231816008
:106AE00041607047B0F90020B0F90210B0F90630EB
:106AF000521A5A4301EBA231818041807047000055
:106B000030B5494B188849490A8A801A85B24848E5
:106B1000484A0F2D047801F150001DD31D880D82C5
:106B2000117A090713D5022C01D0434912E0434DD5
:106B3000B0F90210B5F90050A94205DC02DA01F102
:106B4000020108E0458007E0A1F1020103E0022C08
:106B500002D13B4909884180B0F840101D88691A6C
:106B600089B29C2949D31988A0F84010916A002362
:106B7000B1F5804F31DB3349096DB1F5405F2CDD54
:106B8000314940F26665B1F91010A94212DD43F6B1
:106B90009915A94202DB40F2333108E040F2333567
:106BA000A1F26661694343F2333591FBF5F1A0F838
:106BB000441001E0A0F844302449B2F806510978A5
:106BC000C1F381012DB100BFB0F8441001F21E5194
:106BD0001CE092F84620022A10D0A0F84430022C83
:106BE00001D0A0F84430B0F95C10B0F9443001F1A4
:106BF00014029A420DDAA0F85C2030BD012901D0C0
:106C00000229E1D1B0F8441001F23331A0F8441068
:106C1000E5E703F11402914203DD1439A0F85C109A
:106C200030BDA0F85C3030BD2C07002014000020DF
:106C300023070020AC020020CE040020CC0400205A
:106C4000C80400204801002038050020D00400209E
:106C50002DE9FC4101210220FDF710F90121192045
:106C6000FDF724F901213C48FBF7DEFA4027ADF897
:106C7000007003248DF802400420384D8DF8030085
:106C800069462846FBF77EFAE001ADF800008DF872
:106C900002401C208DF8030069462846FBF772FA73
:106CA0004FF4E0712846FBF7F4FAA815ADF80000A0
:106CB0008DF8024010208DF8030069462848FBF744
:106CC00061FA4FF4A060FCF705FE1D208DF804006A
:106CD00001268DF8056000258DF806508DF80760B7
:106CE00001A8FCF7C5FD1F498C2008801D494FF6FF
:106CF000FA702C3108806E20091F08801948143062
:106D00000680184808300780164920310D80154A42
:106D1000D020121D1080134A45F2F3001832108063
:106D20000A1F45F2500010800E4A4FF6FF703832AD
:106D30001080121D1080121D108041F21B1008805F
:106D400000F012F8FBF722FD064810300580001F06
:106D50000480BDE8FC810000000C1A000010014016
:106D6000000C01400004004070B51D20FCF754FDEC
:106D70002A4D40212846FBF783FA840080212846CB
:106D8000FBF77EFA44EA4004A9152846FBF778FA97
:106D90000443E0B2224C84F83C00FBF7FDFA0546C0
:106DA000052805D91F48C18841F04001C18001E094
:106DB00084F838501C48007A000703D594F838004E
:106DC0001A490D5C4FF6FA702063E062A0626062BF
:106DD0002062E061A0611648606300206064206565
:106DE00084F83F0084F84000FBF784FAA07AFF287B
:106DF00011D0022084F83D000E480088A066284685
:106E0000FBF726FF207820F001002070BDE87040DD
:106E10001D20FCF717BD0120ECE700000010014029
:106E200048010020600A0020AC0200206C98000895
:106E3000DCFF0500240400402DE9F0434E484F4993
:106E400002880B889A1A92B20F2A69D309880180A6
:106E50004B49098B027D00EB42029180017D491C68
:106E6000C9B2017508295BD3002404752246017D4F
:106E700000EB4103491CB3F90430C9B202EB6302D1
:106E800012B201750829F2D33E4904753E4B4A807F
:106E900044800E789D895FEAC67C40F638694FF0E1
:106EA000030714D0A2F22B5C42F6E858C44520D365
:106EB000A1F1020C26F00204ACF8002047750C701A
:106EC00040F22B54A24211DA45F004021EE046F0D3
:106ED00001060E704A4507DD45F001029A8126F051
:106EE00002020A70477519E0447517E045F0020286
:106EF0000CE04A450CDA8775427D12B1521E42758C
:106F00000CE046F002020A7025F007029A8105E0C3
:106F1000B30703D5837D2BB15B1E837540888880C2
:106F2000BDE8F08342F6AA239A4222DAB1F904308E
:106F30002BB941F2CD05AA4201DA4480EEE7134CA9
:106F4000920302EB843241F67244B2FBF4F214B2C3
:106F500040F2333502464480AC4200DA5580B2F943
:106F60000240E41A04F5A374B4F5237FD6D8438015
:106F7000D4E74FF48043FAE7F40A00202C070020FE
:106F8000AC020020E2050020600A0020C8F1FFFFEB
:106F90002DE9F0416D4CDFF8B8E14FF0000594F8B1
:106FA0003410C80706D094F938104B42002958DD38
:106FB0000E4657E0674884F83750A4F84250664AB6
:106FC00090F8380084F840001586CEF80450CEF8CA
:106FD0000850624E40F26663CEF80C50A4F87C3044
:106FE00036F810005E4E768830444FF6FF7606EA9B
:106FF000800024F8300B4FF0806044F8040CA3208C
:10700000208460845810A084E38440F69910208581
:10701000580060854FF48050A08541F23330E08500
:1070200041F26660208641F69910608641F6CC40B8
:10703000A0864FF40050E08642F23330208742F2BF
:107040006660608742F69910A08742F6CC40E087E0
:1070500082F89D5041F00100207184F84450BDE851
:10706000F0811E4694F937004242002801DD0746B0
:1070700000E01746F61B012E0BD0002800DB02466D
:107080005FFA82F684F8380094F84F00012805D0A2
:1070900041E0002900DA1946CEB2F3E794F939301D
:1070A0005942002B01DB184600E0084694F93A20CB
:1070B000C7B25042002A01DB944600E08446BC453A
:1070C00008DD002A00DA0246D7B2002B00DA0B46B0
:1070D000D8B207E0002B00DA0B46DFB2002A00DB53
:1070E0001046C0B204EB4000B0F9501004EB47006A
:1070F00030F9502F11444910018084F84F5084F822
:107100003E5084F83D5084F83C5084F83B5084F85D
:107110003A5084F8395004EB46007546B0F95000F7
:1071200024F8420FBEF80410C82309B26422FDF708
:10713000D5FC6860E968401AA9680844A860B5F9F8
:1071400000104843C013E860608788E7740A002095
:10715000D005002048010020AC0200207E980008E5
:1071600064000020F0B4544890F83410C90776D079
:10717000524990F84030002291F838108B426FD07D
:107180004F4CA0F872204F4DE65C04468E4294F9B5
:10719000374002D0EE5C8E420FD1641C64B280F89E
:1071A0003740EB5C8B4202D1641C80F8374090F989
:1071B00037300F2B1BDD0F2317E0434DEE5C434DA3
:1071C0008E4202D0EE5C8E4211D1641E64B280F811
:1071D0003740EB5C8B4202D1641E80F8374090F957
:1071E00037406FF00E039C4201DA80F83730324BA3
:1071F00090F83F50393390F83740EC5490F83F30D6
:107200005B1CDBB280F83F30062B01D380F83F20B7
:1072100090F9394090F93B309C420ED190F93D40B5
:10722000A3420AD190F93A4090F93C309C4204D1F3
:1072300090F93E40A34200D1012280F84F201F4A1E
:1072400080F8401090F937501378214A012D0DDD58
:1072500014465E07A46804D544F0080403E028E05F
:1072600015E024F00804946080F83510B5F1FF3F74
:107270000ADA5B07936802D523F0080301E043F0C4
:107280000803936080F83510F0BCFBF733B890F832
:107290004F1001290DD1B0F8721043F60953491C63
:1072A00089B2A0F87210994203D9A0F8722080F830
:1072B0004F20F0BC70470000740A002048010020F5
:1072C000609800086698000872980008789800088E
:1072D000AC02002010B5D0E900210369114481FB04
:1072E00003318C0244EA93514260D0E9022382FBCD
:1072F0000332940244EA93521144816010BD0000AD
:1073000030B52049204AB1F86A301088C01A80B2DE
:107310000F2836D31088A1F86A001C4D00204FF0CA
:1073200000432A5C940903D00124B4EB921F24D1BA
:10733000D20622D0164A52F820201268134C12347A
:1073400034F81040224201EB000494F9722008D076
:107350000A2A04DB0A6823FA00F4224308E0521CDC
:1073600009E012F10A0F05DC0A6823FA00F4A243CF
:107370000A6002E0521E84F87220401CC0B211283C
:10738000CFD330BDE80500202C07002074930008FF
:10739000749400082DE9F00779497A480A8903882E
:1073A0009A1A92B2082A74D300880881A1F12C009D
:1073B00042890AB1521E4281734A92F82820802ADB
:1073C00067D302F03F020A70C2890AB1521EC2811D
:1073D000B1F90620902A0CDB8A46FF2A09D08146A3
:1073E000C089002855D1694800230078092805D0B4
:1073F00005E0BDE8F007624800F09AB90823644A46
:1074000092F8EA500DB143F004036248817AC9074B
:1074100001D043F00203D2F808C05FEA0C5101D555
:1074200043F00103176800215B4EFC0302D596F878
:10743000654004B18021C4885FEA446801D541F009
:1074400040015FEA845801D541F020015FEAC47829
:1074500001D041F01001007A400701D541F0080148
:107460004E480078C00701D041F00401A00601D5C4
:1074700041F001010020012D00D1082096F8705044
:1074800085B992F84620022A04D0012A05D03AB1E3
:1074900008E072E040F0030004E040F0020001E088
:1074A00040F001007A0701D440F02000CCF3C00284
:1074B0000025CCF3002C624502D13A0700D4042504
:1074C00096F86F20012A01D145F00105344A0027C2
:1074D000BC4612783E46C2F38102012A04D0022A39
:1074E00004D0032A04D004E0022602E0042600E0CF
:1074F00010262C4A64060ED5214C1C342478240610
:1075000009D51478640606D4274A40F6CC44926D17
:107510006243140C05E0B2F8B62040F699146243B9
:10752000940B4FF008088AF80A804FF061088AF837
:107530000B808AF80C308AF80D108AF80E008AF851
:107540000F508AF81070270A4B4083F069014140C0
:1075500069408AF8117079408AF8124061405246B9
:107560008AF813C071408AF8146051754FF4C871DD
:10757000A9F80E10FF20AAF80600BDE8F007704732
:10758000E80600202C070020E80500202307002043
:10759000AC020020600A0020C00C0020500900202E
:1075A000D0040020480100202008002050488169B4
:1075B00041F0FC0181614FF4A060FCF78BF9FBF70F
:1075C00073F9FCF7EDFAF9F7EBFAFCF7E1F8FDF7E0
:1075D0008BF9FFF73DFBFCF721F8FFF7C5FBFBF745
:1075E000D5F8444D4FF40050A5F81601FEF7C0FD44
:1075F00000214FF4FA5340F2EE220020401C80B2EA
:107600009842FBD3491C89B29142F6D33A480026EE
:1076100080F87260F9F75AF9F9F708FEFCF7F0FA0A
:10762000F9F7CEFCFEF79AFE102234493448F8F7F9
:10763000AAFD01F0DFF9334C344FE08820F0400020
:10764000E0803148017821F020010170FA20F881B2
:107650004FF49670E887FFF7F7F92D492D48FCF7AE
:107660004BFA2D48FCF76EFA2C48416A88472C48A3
:10767000416B8847FEF7DCFF2A48FAF7F7F92A49F9
:107680004220C8802949C8603E71E088E081208995
:10769000208260896082FAF7EDFCFAF74FFCFFF771
:1076A00063F801F047F9FFF7C7FB00F0F9F9FFF7BE
:1076B00027FE01F003F8FEF775F9FAF7ABFAFBF7CE
:1076C000E5FAFFF71DFAFCF7D7FCFAF707FFFAF720
:1076D00039FF00F07BF8FFF75DFE1248FAF78EF8ED
:1076E00000F06AFAFDF744F9FAF7F6F9CDE7000081
:1076F00000100240AC02002038050020C00C002021
:1077000028060020600A00204801002020070020F1
:10771000CC0800209C080020100400203800002025
:10772000E4000020E00900204C0700204404002071
:10773000F0B523490278B0F9064000231F4E31F816
:107740001210FF2C18D0B0F904701E4DBC4231DA73
:1077500000EBE40704F00704BF7AA7408478FFB287
:107760003CB190F801C0ACF1010C64451FDA3C0655
:107770001DD455F822200DE056F822201160124940
:107780008A79521CD2B28A71022A02D38370C380D2
:107790008B71F0BD11608178491CC9B2817042784B
:1077A0009142F6D38370C188491CC180F0BD56F860
:1077B0002220EFE755F822201160F4E754950008E5
:1077C00086930008FC940008BC060020F0B56148D0
:1077D0006149B0F86C200B889A1A92B29C2A7BD32C
:1077E0000988A0F86C105D495D4F91F82A1001F0EE
:1077F000070297F84610022A00D1491E594C80F81A
:107800003E104FF00203E2884FF00001550401D50D
:10781000012236E0A489E50601D5062231E02507DC
:1078200001D508222DE0550603D44F4D2D78AD0625
:1078300001D5042225E0150501D5072221E0150612
:1078400001D50A221DE0950601D50C2219E0150785
:1078500001D50B2215E0550701D4D50501D510221D
:107860000FE0D50601D505220BE0650703D4A50777
:1078700001D4E40702D080F86E3007E0920403D50B
:10788000032280F86E2001E080F86E10374A384CF1
:1078900092F820E0324A251FD2F808C02D4AB2F8EB
:1078A0007060721C92B2BEF1000F0DD02CF4000C6F
:1078B000C7F808C090F86E70B7B11E2F1AD090F8B4
:1078C0006F200AB325E007E04CF40006BE60A0F884
:1078D00070200A2A01D22360F0BD142A01D22B6045
:1078E000F0BDA0F87010F0BD2B60A0F8701080F80B
:1078F0006F10F0BD642E04D2A0F87020322AEED3AF
:10790000E9E7A0F87010EAE77F1C80F86F70A0F834
:10791000701090F86F20012A10D0002AE9D0B0F83A
:107920007060761CB6B2A0F870601E2ED7D32360AC
:107930003C2EDED9521E80F86F20D2E7B0F87020BE
:10794000521C92B2A0F870202360C82AD1D980F8C6
:107950006F10C6E7E80500202C070020C00C0020AF
:10796000AC020020600A002048010020D004002062
:10797000141C0140F0B54248B0F84810491C89B2C7
:10798000A0F8481002297AD33E490024A0F84840C4
:107990000A783D4B042A57D04FF48041082A0BD077
:1079A000A0F10C02B2F900208A4200DA1146B3F9C4
:1079B00080208A4200DA1146344A92698A4200DA0B
:1079C00011B2418282881D8AC2EB8502304D12B20B
:1079D0002D78C5F381062A4D42F291767243B5F9AE
:1079E000765092126A431213C26086681546C6EB3F
:1079F000C60642F3D102F60202EBA6328260C66CE2
:107A00001644C664B0F850707F1CBFB2A0F8507026
:107A1000B7F5806F04D3B6120682A0F85040C46454
:107A2000891A1C4EC26A724340F255564E4302EB0D
:107A30004602466A32444262B3F93030B2EB034F39
:107A400006DD1A04426206E01349B1F90410B3E7F7
:107A5000002A00DA4462C162104990F83D2091F892
:107A600038108A420BD080F83D10B0F84210A0F8D0
:107A70004410B0F84010A0F84210A0F84050F0BDFB
:107A80003805002023070020AC020020580C0020FD
:107A9000D0040020C3F5FFFF740C00204801002033
:107AA00015481649B0F85A200B889A1A92B20F2A34
:107AB00020D30988A0F85A10B0F9001041F63022FE
:107AC00051438913A0F86C100D494FF480420B7894
:107AD000A0F10C01022B06D1B1F90030934202DA79
:107AE0001B1D0B8000E00A800021A0F8601020F828
:107AF0005C1F428070470000380500202C070020E2
:107B0000230700204FF6FF7202EA800210F4404380
:107B100015480ED0B3F5804F14D0B3F5004F4FEA9F
:107B2000122216D0C2F5807330F813305B424B80BE
:107B300005E0120A30F812304B80C2F5807230F83E
:107B400012000FE0120AC2F5807330F813304B8038
:107B500005E030F81230C2F580725B424B8030F89D
:107B6000120040420880704770910008104A518A04
:107B7000908AD28A16384639A2F1110200D54942BC
:107B8000002A00DA52421144002800DA4042084438
:107B9000084943F6284300B2B1F936205A439213FC
:107BA00040F2D733584302EBA030C886704700003C
:107BB000AC02002038050020F0B5904990480A89B1
:107BC00003889A1A92B23E2A1ED30088088101F1D6
:107BD00038004FF4FA63428A9A4202D2521C42821F
:107BE00000E04382874A92F82220802A0CD302F0D8
:107BF0003F020A70B1F90620402A06DBFF2A04D0B2
:107C0000C2883AB1521EC280F0BDBDE8F0407B4848
:107C1000FFF78EBD428A9A42F6D307784FF0010EE5
:107C20003A074FF0FF055BD5847A40F2DC526307D8
:107C300008D444F004038372C28081F80BE081F819
:107C40000AE04CE04378072B05D0032B03D0052B2B
:107C500001D0062B07D1660605D444F04003837299
:107C6000C280052239E0654A5FEA437C02F13802AE
:107C70004FF42076127A0DD55FEAC26C0AD45FEA1F
:107C8000446C07D442F0100202723A0628D4C6802F
:107C9000192222E0DF0709D0970707D4670605D429
:107CA00042F002020272C680042216E09F0709D544
:107CB000170707D4670605D442F008020272C6808F
:107CC00003220AE01B070BD5530709D4630607D428
:107CD00042F004020272C6800B22CA728A72CD8000
:107CE000494AB2F92230B2F91A7003F23D14002267
:107CF000A74200DB0276414E444C06F13806A479D7
:107D0000B6895FEAC46C06F101064FF4C874B6B2D6
:107D100013D58681B6F57A7F05D9017A21F08001E5
:107D200001728281F0BD037A1E06FBD4828143F08A
:107D300080020272C480112035E09F4216DA037E71
:107D4000052B13D28681B6F5487F04D98281027A49
:107D500022F040020272027A5606E3D45B1C0376DC
:107D600042F040020272C48002201CE0284B1C89B1
:107D7000C4F3C006C4F3002740F2EE24BE4216D17D
:107D80001E78360713D4427E012ACBD1428BB2F53E
:107D9000167F02D2521C4283F0BD827A42F0020268
:107DA0008272C4800F20C8728872CD80F0BD93F8B3
:107DB0000D714FF40046012F18D1164F41F6583C73
:107DC0007F6C674512DD83F80CE1134B1E60C38A9C
:107DD000A34202D25B1CC382F0BD4FF4FA73C3808E
:107DE0001C23CB728B72CD80C282F0BDC2820A4846
:107DF00083F80C21001F0660F0BD0000CC060020B7
:107E00002C070020E8050020D0040020600A002094
:107E1000AC02002048010020140801402DE9F05F69
:107E2000FE48FF49DFF8FCA3007E0A1D131D012850
:107E300050465AD030F85A4F0C8041881180BAF819
:107E40005E001880FDF746FEF74DF84C49F2CD3242
:107E5000B5F91E106183B5F9200043F6CC4C01EB57
:107E6000400050430014A083B4F92230B4F92060DC
:107E700000FB03F201FB062242F38F326282B4F967
:107E8000167007FB0CF7BF1340F2333C704302FB44
:107E90000CF201FB130007EBA232E28240F38F30B9
:107EA000A082B4F91810E24FC1EBC10141F3D10136
:107EB00001EBE000DF4E2083786C306031693046A2
:107EC0008847DD49308948800846FDF7E5FEDFF840
:107ED0006CB301264FF000099BF8000008280CD075
:107EE000618F218204284AD01AE030F8604F0C805C
:107EF00041881180BAF86400A3E7D14890F937109F
:107F0000491C022939D890F8741019B1B4F85A00F4
:107F1000208205E0618F2182A4F85A1080F87460F5
:107F2000B4F91410B4F90A00C64AF9F7B9FAE062D4
:107F3000BAF91611884204DDC248E162027C914020
:107F40008162BA48DFF800E3503847F2A3080278AC
:107F50004EF24611002A7AD0012A79D080F800909A
:107F60009BF8000004280DD0B64AB4F91210B4F9F9
:107F70000800303AF9F794FA08E0608FC8E7686AB9
:107F80000014E062B87A002863D0B048A3462546C2
:107F9000A062AC4C443C2060E86A6060204610352A
:107FA000FCF744F8A14928883C39FFF7ABFDDFF81E
:107FB0007C82A8F15008D8F81410C8F87010B5F9F0
:107FC0001010A068B5F9122000FB01F7E3685043D8
:107FD00003FB127444F38F3703FB0100AF8740F3B8
:107FE0008F34EC879A4D28466F80AC80FEF728FAD4
:107FF000287F08F11805012871D0604241104DF624
:10800000B350474369803A142A804046A8F8044098
:108010008B18C380891AA8F808108AF80C90B8F950
:1080200004305446002B00DD2673B8F90600002802
:1080300002DD217B891C2173B8F90820002A02DDAA
:10804000217B091D2173217B072979D202E007E0FA
:108050002CE05AE0DFE801F07470886E84728600CC
:10806000B5F91E2042448A420AD8B5F9202042447C
:108070008A4205D8B5F9222042448A427FF670AF81
:10808000A0F80290B7F8B6204946B2F5C87F01D8EB
:10809000467006E0B2F5487F01D8022200E00322D4
:1080A00042708AF80F108BF8001025E080F80090DD
:1080B000B5F91EC04A46C4448C4509D8B5F920C05C
:1080C000C4448C4504D8B5F9225045448D42D5D9D5
:1080D000B7F8B610B1F5C87F02D8467007E017E0D0
:1080E000B1F5487F01D8022100E0032141704280B0
:1080F0008AF80F208BF80020BEF8061041F40061CA
:10810000AEF80610F9F70CFF2AE74FF4AF703DE721
:108110004F484DF6B352B0F92030594249106980AA
:10812000B0F91E00504302142A804046A8F80430DB
:108130006EE705E0667303E0022100E0032161734E
:108140009BF80010434E0129434F617BDA460DD066
:10815000072961D2DFE801F060FDFCFBFAF9F800C5
:108160000421ECE70521EAE70621E8E70729F0D238
:10817000DFE801F052042980A5D3F000014618463B
:10818000FBF7A0FC2860B5F9020040F68151484396
:1081900080136880B5F9001040F68152514389136D
:1081A00029804218A2F68152B8F80E305242C3EB31
:1081B000620212B2A8F80C20002A01DCA8F80C9088
:1081C000B8F80C206EE1404201B2504200B2FBF719
:1081D00079FC2860B5F9020040F6815148438013CC
:1081E0006880B5F9001040F6815251438913298007
:1081F0004218A2F68152B8F80E305242C3EB620226
:1082000012B2A8F80C20002A01DCA8F80C90B8F8EB
:108210000C20A4F85E2021E0E9E00000E009002045
:10822000342C0140AC0200203805002064000020FE
:1082300048010020440400200004002023070020FF
:10824000740A0020CC080020600A0020A2FEFFFF74
:10825000140A002000240140002801401044A4F822
:108260005A00084452E13046F8F7F8FC01231A4658
:108270000721B1E019461046FBF724FC2860B5F948
:10828000020040F68151484380136880B5F9001020
:1082900040F681525143891329804218A2F6815237
:1082A000B8F80E305242C3EB620212B2A8F80C20AA
:1082B000002A01DCA8F80C90B8F80C204DE15942D6
:1082C000404209B200B2FBF7FDFB2860B5F902009D
:1082D00040F68151484380136880B5F9001040F69C
:1082E00081525143891329804218A2F68152B8F86D
:1082F0000E305242C3EB620212B2A8F80C20002AE0
:1083000001DCA8F80C90B8F80C2056E13046F8F7DC
:10831000A5FC01231A4605215EE01146FBF7D2FBBE
:108320002860B5F9020040F6815148438013688007
:10833000B5F9001040F68152514389134218A2F654
:1083400081522980524206E076E14AE11BE1ECE0ED
:10835000BCE08FE013E0B8F80E30C3EB620212B25B
:10836000A8F80C20002A01DCA8F80C90B8F80C2022
:10837000A4F85C201044A4F85A0008444EE150428E
:1083800001B2584200B2FBF79DFB2860B5F902002C
:1083900040F68151484380136880B5F9001040F6DB
:1083A00081525143891329804218A2F68152B8F8AC
:1083B0000E305242C3EB620212B2A8F80C20002A1F
:1083C00001DCA8F80C90B8F80C204FE13046F8F723
:1083D00045FC01231A4606213846F8F73FFC0121E7
:1083E0003046F8F7B1FB01213846F8F7ADFBB04E47
:1083F000BAF8080055463080BAF80A007080BAF81A
:108400001000B0803046F9F745FAB4F85A00F18808
:108410000844A4F86000B4F85C0031890844A4F86A
:108420006200B4F85E0071890844A4F86400317EEB
:10843000A048012978D034F85A1F01806188418012
:10844000A18881809B49028808310A8042884A803D
:10845000808888809748896A0830884795F83E0068
:1084600000287DD0F8F7FEFD15F83E0F401E28705D
:10847000BDE8F09F01461846FBF724FB2860B5F9DC
:10848000020040F68151484380136880B5F900101E
:1084900040F68152514389134218A2F6815252424A
:1084A00029805208A4F85E201044A4F85C00084417
:1084B000A4F85A0000213046F8F746FB0021384660
:1084C000F8F742FB01231A460621CCE6404201B2EE
:1084D000504200B2FBF7F6FA2860B5F9020040F608
:1084E0008151484381136980B5F9000040F68152FB
:1084F000504380130A18A2F6815252425208288033
:108500001144A4F85E20A4F85A100844A4F85C00B2
:1085100000213046F8F718FB00213846F8F714FB25
:1085200001231A4605219EE6B4E019461046FBF7E2
:10853000C9FA2860B5F9020040F68151484380131A
:108540006880B5F9001040F68152514389134218F2
:10855000A2F68152524229805208A4F85A2000E023
:108560009BE01044A4F85E000844A4F85C000021DD
:108570003046F8F7E9FA00213846F8F7E5FA012322
:108580001A460721C2E65942404209B200B2FBF73F
:1085900099FA2860B5F9020040F6815148438013EA
:1085A0006880B5F9001040F6815251438913421892
:1085B000A2F68152524229805208A4F85A2010444F
:1085C000A4F85C000844A4F85E0000213046F8F7E7
:1085D000BBFA00213846F8F7B7FA01231A460621FC
:1085E00094E61146FBF76EFA2860B5F9020040F6F2
:1085F0008151484381136980B5F9000040F68152EA
:10860000504380130A18A2F6815252425208288021
:108610001144A4F85C20A4F85A100844A4F85E00A1
:1086200000213046F8F790FA00213846F8F78CFA26
:1086300001231A460521C9E6504201B2584200B250
:10864000FBF740FA2860B5F9020040F68151484333
:1086500080136880B5F9001040F6815251438913A8
:108660004218A2F68152524229805208A4F85C2096
:108670001044A4F85E000844A4F85A0000213046D3
:10868000F8F762FA00213846F8F75EFA01231A4635
:1086900007219BE634F8601FCFE607480088A0F565
:1086A000D04168393FF4E4AEBDE8F05FF9F786BB2E
:1086B000E009002030000020182C01402DE9F04195
:1086C000904C9148B4F862100288511A89B20F296F
:1086D0006FD30088A4F862008C480088DFF83082ED
:1086E000C0074FF000054FF0010741D0874AD4E999
:1086F0000C1024321388B1EB530F02D21288511A96
:1087000008444FF4F371884200D208468149B1FB16
:10871000F0F0616CC1F35101084406466064F7F75C
:108720007CFE00227C4BF7F7E4FD4FF040427B4B90
:10873000F7F7DFFD0E22F7F74BFEF7F7A5FEA4F8DB
:10874000AC0094F86D00401CC0B284F86D0008289D
:1087500034D36C4898F84620001F03789A4201D021
:10876000027045806E4A13786E4A23B1458021E03D
:108770006564256558E0D8F89410A1F5FA618E4239
:1087800011DDE16D8B1C9E4205DDB0F902100A2956
:108790000DDA491C06E08E4205DAB0F90210002914
:1087A00008DD491E4180B0F902000A2802DB17707B
:1087B00001E0A2E01570E66584F86D505A484FF468
:1087C000A5420178C1F38101012949D002294AD08B
:1087D00044F687712181A4F8A820B0F9243089B229
:1087E0004B439B13A4F8A430B0F90E000023704350
:1087F000B0FBF1F0216DC0F3D100C1EBC101C902A2
:1088000000EB91302065F017810341EA9641B003F7
:10881000F7F788FCB4F8AA10C1EBC101C902C0087F
:1088200000EB9130A4F8AA00616C206F0844206727
:1088300094F87420521CD2B284F87420082A05D30C
:10884000C008A4F8760084F8745025673748384E7D
:10885000C3885A0633D498F80F20022A06D02CE099
:1088600043F20451B6E744F24621B3E7B26840F65A
:108870009916B24221DD94F8382094F88E60B24205
:108880000CD084F88E2094F83D2002F00106C2F34B
:108890004002964202D1A4F88A5004E0B4F88A203B
:1088A000B2F5966F05D2B4F88A00401CA4F88A008D
:1088B00005E043F08002C28001E0A4F88A5011482C
:1088C00094F83F30B8300C2B01D2C57400E0C77467
:1088D000174A0F4C41F2482692F83C20B4F88240E7
:1088E00041F2504C0C2B0AD3B14208DB012A06D0CE
:1088F000614502DD002C00D18774BDE8F0818574EC
:10890000FBE70000480100202C0700200004004085
:10891000AC0200204564BD0100209C40133B334065
:10892000FE030020FF030020D0040020600A002086
:108930003805002070B5284C284821880288511A33
:1089400089B23E2947D3008820802548808B254D59
:10895000800228606969284688472349A868FDF78E
:1089600077F822496060CB885A072ED40022B0F1F4
:10897000F05F0FD9E089B0F5FA7F08D943F0040021
:10898000C8801B48017821F0020101701CE0401CE6
:10899000E0811AE0B0F1D25F0CD94FF4F031A1EBD5
:1089A00010308003C910B0FBF1F0206100280CDA10
:1089B00022610AE0B0F1C85F03D94FF48040206122
:1089C00003E023F00400C880E281D4E90401884276
:1089D00000DB0846A06170BD580C00202C07002069
:1089E000AC0200209406002068970008600A00206E
:1089F000E205002005494FF4804048610861886124
:108A00000348C18821F48271C1807047580C00204E
:108A1000600A00202DE9F041384C394E394F20785A
:108A200041F23331C2074FF000050CD0A28962B386
:108A300094F90700002800DA4042C0B2032829D286
:108A400040F2AE702AE0A570E5732F4AE571A5816A
:108A500092F83830237220F00800A18040F0020024
:108A600020703D867560B560F560116D490005D0D8
:108A700041F68461A18140F010002070C0B240F046
:108A8000010020706574BDE8F081658120F0100060
:108A9000207015E0042803D240F6510060810FE0F9
:108AA000052802D240F69910F8E740F6CC42062895
:108AB00003D3072801D3082801D2628100E0618135
:108AC00097F89D0098B9B088102301B2B4F90A0054
:108AD0003622FCF703F87060F168401AB168084468
:108AE000B060B6F900104843C013F0603886388E85
:108AF00010B10120A070C6E7A570C4E7740C002077
:108B0000AC060020AC020020480100202DE9F04115
:108B1000554C2678F0077CD05448217A544D90F873
:108B2000380081427BD0534A2346DFF84CC1575C62
:108B300093F90E2093F90730874203D01CF8017097
:108B4000874213D146F002065B1C26705BB2E371CC
:108B50001CF80110814201D15B1CE37194F90710EC
:108B6000062901DD0621E171521C1CE0434F17F874
:108B700001C0434F844503D017F801C0844513D189
:108B800026F002065B1E26705BB2E371795C8142BF
:108B900001D15B1EE37194F907306FF005018B4240
:108BA00000DAE171521EA273207294F907108A1C38
:108BB000042A02D941F68462A2812C4A0129127842
:108BC0000ADD2B4B56079B6802D543F0080301E0F2
:108BD00023F00803AB606070B1F1FF3F09DA510781
:108BE000A96802D521F0080101E041F00801A9605F
:108BF0006070F9F77FFBA078012810D121488068C8
:108C0000A3280CDA94F90700022803DD0220E071A2
:108C100005E01EE06FF00101884200DAE171A089F1
:108C2000002630B1401E0004000CA08101D1E67185
:108C3000A673E87B04280CD0B5F9301051234122EB
:108C40000020FBF74BFF2886002802D1E07B10B103
:108C5000A670BDE8F0810C4806700C4806702078BC
:108C600020F001002070F4E7740C0020480100207F
:108C7000AC0200206098000866980008729800080E
:108C800078980008380500204007002023070020BE
:108C9000743F713D9B3BED396238F436A135653444
:108CA0003F332A32273133304C2F722EA32DDF2C45
:108CB000242C722B000000361C070038AA0A003A48
:108CC000AA0A003CCC0C003ECC0C0040380E0042FE
:108CD000380E0044380E0046380E0048380E004A60
:108CE000C711004CC711004EC7110050C7110052E8
:108CF000C7110054C7110056C7110058C711005AB8
:108D0000C711005CC711005EC7110060C711006287
:108D1000C7110064C7110066C7110068C711006A57
:108D200000000036220200388E03003AB005003CF5
:108D3000D207003EF4090040160C0042380E0044F1
:108D40005B100046C71100483313004A9F14004CC3
:108D50009F14004E0B1600507717005277170054DF
:108D600077170056771700587717005A7717005C67
:108D70007717005E77170060771700627717006437
:108D800077170066771700687717006A00000036CB
:108D900000000038B600003A6C01003C2202003EA0
:108DA000D80200408E03004244040044FA04004606
:108DB000B00500486606004A1C07004CD207004E6A
:108DC000880800503E090052F4090054AA0A0056CF
:108DD000600B0058160C005ACC0C005C820D005E33
:108DE000380E0060EE0E0062A40F00645B10006697
:108DF00011110068C711006A00000034000000363D
:108E0000000000380000003A0000003C0000003E76
:108E10000000004000000042000000440000004646
:108E2000000000480000004A0000004C0000004E16
:108E300000000050000000520000005400000056E6
:108E4000000000580000005A0000005C0000005EB6
:108E50000000006000000062000000640000006686
:108E60000000006844145858587011115858587030
:108E700041115858487011144858587014115848E6
:108E8000587000200072002000700020006E00204A
:108E9000006C0020006A00200068002000660020AE
:108EA000006400200062002000600020005E0020BE
:108EB000005C0020005A00200058002000560020CE
:108EC000005400200052002000500020004E0020DE
:108ED000004CA320004AA320004847210046EB2174
:108EE0000044EB2100428F2200408F22003E7A2472
:108EF000003C7A24003A66260038512800343D2A86
:108F00000030702D002CA33000287A340024513812
:108F10000020CC3C001C0040001800400014004021
:108F200000100040000C0040000800400004004019
:108F30000000000001020304050005000102030413
:108F40000104000305020000F001000036010000EA
:108F5000F8000000BA0000007C0000007C00000067
:108F60007C00000041141411111444111414411117
:108F70000000290052007B00A400CC00F5001E0177
:108F8000470170019901C201EA0113023C02650226
:108F90008E02B602DF020803300359038203AA03DC
:108FA000D303FB0324044C0475049D04C504EE04A0
:108FB00016053E0567058F05B705DF0507062F0671
:108FC00057067F06A706CE06F6061E0746076D075C
:108FD0009507BC07E4070B08320859088108A80860
:108FE000CF08F6081D0944096A099109B809DE0984
:108FF000050A2B0A520A780A9E0AC40AEA0A100BCA
:10900000360B5C0B820BA80BCD0BF30B180C3E0C34
:10901000630C880CAD0CD20CF70C1C0D410D650DCA
:109020008A0DAF0DD30DF70D1C0E400E640E880E89
:10903000AC0ECF0EF30E170F3A0F5E0F810FA40F79
:10904000C70FEA0F0D103010531075109810BA109A
:10905000DD10FF102111431165118711A911CA11EB
:10906000EC110D122E12501271129212B312D41270
:10907000F41215133613561376139613B713D7132A
:10908000F61316143614561475149414B414D31419
:10909000F214111530154E156D158C15AA15C8153D
:1090A000E7150516231641165F167C169A16B71695
:1090B000D516F2160F172C17491766178317A01726
:1090C000BC17D917F51711182E184A1866188118E9
:1090D0009D18B918D418F0180B19261942195D19E2
:1090E00078199219AD19C819E219FD19171A311A10
:1090F0004C1A661A801A991AB31ACD1AE61A001B6E
:10910000191B331B4C1B651B7E1B971BAF1BC81BFE
:10911000E11BF91B121C2A1C421C5A1C721C8A1CC3
:10912000A21CBA1CD21CE91C011D181D301D471DB4
:109130005E1D751D8C1DA31DBA1DD01DE71DFD1DD7
:10914000141E2A1E401E571E6D1E831E981EAE1E24
:10915000C41EDA1EEF1E051F1A1F2F1F451F5A1FA0
:109160006F1F841F991FAE1FC21FD71FEC1F002047
:1091700000006400C9002D019201F7015B02C002EA
:1091800024038903ED035204B6041A057F05E305A1
:109190004706AB060F077307D7073B089F0802096E
:1091A0006609C9092D0A900AF30A560BB90B1C0C63
:1091B0007F0CE20C440DA60D090E6B0ECD0E2F0F89
:1091C000900FF20F5310B41015117611D7113812F9
:1091D0009812F8125813B81318147714D6143515BA
:1091E0009415F3155116B0160E176B17C9172618DC
:1091F0008318E0183D199919F519511AAD1A081B71
:10920000631BBE1B181C731CCD1C261D801DD91D85
:10921000321E8A1EE31E3B1F921FEA1F4120982028
:10922000EE2044219A21EF2145229922EE22422369
:109230009623E9233C248F24E22434258525D72551
:1092400028267826C82618276827B72706285428EE
:10925000A228EF283D298929D629222A6D2AB82A51
:10926000032B4D2B972BE12B2A2C722CBB2C022D80
:109270004A2D912DD72D1D2E632EA82EEC2E302F8A
:10928000742FB82FFA2F3D307F30C030013141317B
:109290008131C13100323F327D32BA32F73234335C
:1092A0007033AC33E73322345C349534CE34073535
:1092B0003F357735AE35E4351A3650368536B93612
:1092C000ED36203753378637B737E93719384938FD
:1092D0007938A838D738053932395F398B39B739F9
:1092E000E2390D3A373A603A893AB23ADA3A013B12
:1092F000283B4E3B733B983BBD3BE03B043C263C4C
:10930000483C6A3C8B3CAB3CCB3CEA3C093D273DAE
:10931000443D613D7D3D993DB43DCE3DE83D013E3E
:109320001A3E323E493E603E763E8C3EA13EB53E00
:10933000C93EDC3EEF3E013F123F233F333F433FF8
:10934000513F603F6E3F7B3F873F933F9E3FA93F2A
:10935000B33FBC3FC53FCD3FD53FDC3FE23FE83F99
:10936000ED3FF13FF53FF93FFB3FFD3FFF3FFF3F43
:10937000FF3F0000E7382C35002020EF2037202366
:109380003320262021000080020004000800100085
:10939000000200040008040000020004000800109D
:1093A0000020004000800400000000800000004019
:1093B0000000002000000010000000080000000471
:1093C00000000002000000010000800000004000DA
:1093D0000000200000001000000008000000040051
:1093E00000000200000001000080000000080140B1
:1093F000000C0140000C0140000C0140000C014039
:10940000000C0140000C0140000C01400010014024
:109410000010014000100140001001400010014008
:1094200000100140001001400010014000140140F4
:1094300004080140040C0140040C0140040C0140EC
:10944000040C0140040C0140040C0140040C0140D8
:1094500004100140041001400410014004100140B8
:1094600004100140041001400410014004100140A8
:109470000414014008080140080C0140080C014098
:10948000080C0140080C0140080C0140080C014088
:10949000080C01400810014008100140081001406C
:1094A0000810014008100140081001400810014058
:1094B00008100140081401400C0801400C0C014048
:1094C0000C0C01400C0C01400C0C01400C0C014038
:1094D0000C0C01400C0C01400C1001400C10014020
:1094E0000C1001400C1001400C1001400C10014008
:1094F0000C1001400C1001400C14014010080140F8
:10950000100C0140100C0140100C0140100C0140E7
:10951000100C0140100C0140100C014010100140D3
:1095200010100140101001401010014010100140B7
:1095300010100140101001401010014010140140A3
:10954000000000000000000000000000000000001B
:109550000000000014080140140C0140140C0140EC
:10956000140C0140140C0140140C0140140C014077
:10957000140C01401410014014100140141001405B
:109580001410014014100140141001401410014047
:1095900014100140141401400000000000000000FD
:1095A000000000000000000000000000FFFFFF0FAF
:1095B0000FFFFFFFFFF0FFFFFF0FFFFFFFFFF0FFB9
:1095C0000FFFFFFFFFF0FFFFFF0FFFFFFFF0FFFFA9
:1095D0000FFFFFFFFFF0FFFFFF0FFFFFFFFFF0FF99
:1095E000FFFF0FFFFFFFFFF0FFFFFF0FFFF0FFFF89
:1095F00000000040400000000004000000400000A7
:1096000000000400400000000004000000400000D2
:1096100000040000400000000004000000400000C2
:1096200000000400000040000000000400000040B2
:10963000000400000000008080000000000800001E
:10964000008000000000080080000000000800000A
:1096500000800000000800008000000000080000FA
:1096600000800000000008000000800000000008EA
:109670000000008000080000000000202000000022
:109680000002000000200000000002002000000096
:109690000002000000200000000200002000000086
:1096A0000002000000200000000002000000200076
:1096B0000000000200000020000200000000006026
:1096C00060000000000600000060000000000600CE
:1096D00060000000000600000060000000060000BE
:1096E00060000000000600000060000000000600AE
:1096F000000060000000000600000060000600009E
:1097000000800200040008001000000200040008AD
:109710000400000200040008001000200040008047
:1097200004000000FF7FFFFFFDFFFFFFFBFFFFFFC7
:10973000F7FFFFFFEFFFFFFFFFFDFFFFFFFBFFFF57
:10974000FFF7FFFFFBFFFFFFFFFDFFFFFFFBFFFF3B
:10975000FFF7FFFFFFEFFFFFFFDFFFFFFFBFFFFF91
:10976000FF7FFFFFFBFFFFFF0000401F7A19030090
:109770000000001E897603000000C01C3BDF0300D0
:109780000000801BD15704000000401A9FE0040035
:10979000000000199E7B05000000C017E42C0600A5
:1097A000000080160DF806000000401593DE07004B
:1097B0000000001408E608000000C012B1110A0001
:1097C0000000801101650B0000004010E6E30C0072
:1097D0000000000F46940E000000C00D46771000F8
:1097E0000000800CB08F12000000400BD2DE14008D
:1097F0000000000A5E6317000000C008601A1A002B
:109800000000800726FC1C0000004006000020002D
:10981000000000057A1923000000C003D539260096
:10982000000080025851290000004001764F2C00B2
:109830000000000046252F000000C0FE2AC63100AF
:10984000000080FDA1283400000000FB4B1F380001
:10985000000080F829053B00000000F6EFFE3C0008
:1098600001020304050002030405000103040500CE
:10987000010205000102030404050001020355056D
:109880000010AA1A55250030AA3A0000AA0A551558
:109890000020AA2A5535FF3FB89800080000002094
:1098A00058070000E4060008B49900085807002093
:1098B000E00900005867000845020406082D01026F
:1098C00003040405480607080913392B1B084D0437
:1098D000211355152A4006190801A713873D1B08B7
:1098E000AD041AA70401251702060405010314801C
:1098F00020FF8BAA0A0201A415AA0A5515000859CF
:1099000020AA2A5535FF3F07290301050406020353
:10991000127C1573FFFF04FF8080010129025F6440
:1099200002130A13D16A12081201100C0504060270
:1099300003010103070505280B01020304020607C2
:109940000303040C3D0706040509191F1919043106
:109950000506064BAA1A024B381E026910312E402A
:10996000FD3969260211042F405F020C26405B2658
:109970002ACD55155515123902017F0316D0071A45
:10998000FF01013B0261AA0C12080108A8147F998B
:109990003F23403313D5720A1608DC9122031210BC
:1099A0000A17401C12600A16901B014D13E56A024B
:0499B00000080000AB
:020000040800F2
:10FC00004A46545A594D46312D4E3330202020203B
:10FC1000050406020301AA0AAA0AAA0AAA0AAA0A4B
:10FC2000AA0ADE3F00100000FF0131000201664613
:10FC300000400040513800400040004000400101B9
:10FC400000400040FF387B257B257B25FF003333B8
:10FC50000201401F00016626B81E6626FFFFFFFF57
:10FC6000FFFF01010100010000000300000200008D
:04FC70000000AA5591
:04000005080000ED02
:00000001FF
